:020000040000FA
:3C000000FFFF627515FFFFFFFFFFFFFFFFFFFFFFFFFFFFFFFFFFFFFFFFFFFFFFFFFFFFFFFFFFFFFFFFFFFFFFFFFFFFFFFFFFFFFFFFFFFFFFFFFFFFFFFFFFFFFF11
:3C003C000000000084800000000000000000000008C20800001000420800080000000000000000000004000000040004000004840000004808000848000012FF0B
:3C007800000004000000000000000000000000000400040004800080040004000000000000000000008004000480008004000000000000800400048000009EFE04
:3C00B4000000000000000000000004800000000000000000000000000000000000000000000004000400000000000000000000000080040000000000000092FE70
:3C00F00000008C808CC004800480008004800480048204820CD0048004820482048004800480008004A0148414A404A0148414A404000480048804880000DCFF05
:3C012C0000000C800C810480048004C2048004801481148084C084C00C801480048004800480048004C2048004C18480148014A204A10C8204801484000082FE9B
:3C016800000004000480000000000480000000000480040004800080040004000000000000000400048004000480008004000480008004800400048000001AFEFF
:3C01A400000004800480048004800480048004800480048004800480048004800480048004800480048004800480048004800480048004800480048000001EFE17
:3C01E000000000848020048004808C8004800480002400825000040000810084048004800480148214040882100204200084000404800448088100440000DCFEAB
:3C021C000000000000000000000000000000000000000000000000000000000000000000000000000000000000000000000000000084060000000000004838FE9E
:3C0258000000000000000000000000000000000000000000000000000000000000000000000000000000000000000000000000000000060000000000000078FEEE
:3C02940000000000000000000000000000000000000000000000000000000000000000000000000000000000000000000000000000800200000000000000BCFEF2
:3C02D0008A000000000000000000000000000000000000000000000000000000000000000000000000000000000000000000000000C05200000000000000D1FE87
:3C030C0002000000000000000000000000000000000000000000000000000000000000000000000000000000000000000000000000800400000000000001FBFF34
:3C034800020000000000000000000000000000000000000000000000000000000000000000000000000000000000000000000000000002000000000000000DFF69
:3C03840002000000000000000000000000000000000000000000000000000000000000000000000000000000000000000000000000800000000000000000AFFF0D
:3C03C00008020000000000000000000000000000000000000000000000000000000000000000000000000000000000000000000000004800000000800120B2FF5D
:3C03FC000000000000000000000000000000000000000000000000000000000000000000000000000000000000000000000000008080060000000000000070FE51
:3C0438000000000000000000000000000000000000000000000000000000000000000000000000000000000000000000000000000000060000000000000078FE0C
:3C04740000000000000000000000000000000000000000000000000000000000000000000000000000000000000000000000000000800200000000000000BCFE10
:3C04B00002000000000000000000000000000000000000000000000000000000000000000000000000000000000000000000000000C05200000000000000D9FE25
:3C04EC0002000000000000000000000000000000000000000000000000000000000000000000000000000000000000000000000000800400000000000000EBFF64
:3C052800000000000000000000000000000000000000000000000000000000000000000000000000000000000000000000000000000002000000000000003CFE5B
:3C05640002000000000000000100000001000000000000000000000000000000000000000100000000000000000000000000000001800000010000000100BFFF15
:3C05A00002000000000000800000008000000000000000000000000000000000000000800000008001000000000000000000008000002880000000800000B5FFC0
:3C05DC0000000000000000000000000000000000000000000000000000000000000000000000000000000000000000000000000000C10A00000000000048A0FF31
:3C061800000000000000000000000000000000000000000000000000000000000000000000000000000000000000000000000000000002000000000000003CFE6A
:3C06540000000000000000000000000000000000000000000000000000000000000000000000000000000000000000000000000000800200000000000000BCFE2E
:3C0690008A00000000000000000000000000000000000000000000000000000000000000000000000000000000000000000000000080220000000000000087FF7C
:3C06CC0012000000000000000000000000000000000000000000000000000000000000000000000000000000000000000000000000800000000000000044ABFE73
:3C070800020000000000000000000000000000000000000000000000000000000000000000000000000000000000000000000000000000000000000000002FFF85
:3C07440002000000000000000000000000000000000000000000000000000000000000000000000000000000000000000000000000800600000000000000C9FF29
:3C07800000080000000000000000000000000000000000000000000000000000000000000000000000000000000000000000000000001608000000000000E0FF38
:3C07BC0000000000000000000000000000000000000000000000000000000000000000000000000000000000000000000000000000A4160000000000004808FFF8
:3C07F8000000000000000000000000000000000000000000000000000000000000000000000000000000000000000000000000000000060000000000000078FE49
:3C08340000000000000000000000000000000000000000000000000000000000000000000000000000000000000000000000000000800200000000000000BCFE4C
:3C0870008A00000000000000000000000000000000000000000000000000000000000000000000000000000000000000000000000080220000000000000087FF9A
:3C08AC00020000000000000000000000000000000000000000000000000000000000000000000000000000000000000000000000008000000000000000082FFF58
:3C08E800020000000000000000000000000000000000000000000000000000000000000000000000000000000000000000000000000000000000000000002FFFA4
:3C092400020000000000000000000000000000000000000000000000000000000000000000000100000000000000000000000000018002000000000000008DFE86
:3C09600010040000000000000000000000000000000000000000000000000000008001000080000000000000000000000000008000808D0000000080012064FFB5
:3C099C0000000000000000000000000000000000000000000000000000000000000000000000000000000000000000000000000000A206000000000000481EFE13
:3C09D8000000000000000000000000000000000000000000000000000000000000000000000000000000000000000000000000000000060000000000000078FE67
:3C0A140000000000000000000000000000000000000000000000000000000000000000000000000000000000000000000000000000800200000000000000BCFE6A
:3C0A50008A00000000000000000000000000000000000000000000000000000000000000000000000000000000000000000000000080320000000000000097FE99
:3C0A8C000A0000000000000000000000000000000000000000000000000000000000000000000000000000000000000000000000008000000000000040406FFFB6
:3C0AC800020000000000000000000000000000000000000000000000000000000000000000000000000000000000000000000000000000000000000000002FFFC2
:3C0B0400020000000000000001000000010000000000000000000000000001000000000000000000000000000000000000000000008002000100000001008DFFA0
:3C0B400000080000000000800000008000000000000000000000000000800000000000000000000000000000000000000000000000008C80000000800000D2FE95
:3C0B7C0000000000000000000000000000000000000000000000000000000000000000000000000000000000000000000000000000900200000000000000ACFE01
:3C0BB80000000000000000000000000000000000000000000000000000000000000000800000000000000000000000000000000000000200000000000000BCFEC5
:3C0BF40000000000000000000000000000000000000000000000000000000000000000000000000000000000000000000000000000800600000000000000F8FE49
:3C0C30008A000000000000000000000000000000000000000000000000000000000000000000000000000000000000000000000000A05600000000000000F5FE15
:3C0C6C000200000000000000000000000000000000000000000000000000000000000000000000000000000000000000000000000080080000000000000027FF9C
:3C0CA800020000000000000000000000000000000000000000000000000000000000000000000000000000000000000000000000000000000000000000003EFED2
:3C0CE40002000000000000000000000000000000000000000000000000000000000000000000000000000000000000000000000000800400000000000000EBFF64
:3C0D200010080000000000000000000000000000000000000000000000000000000000800000000000000000000000000000000000000204000000000000E5FE16
:3C0D5C0000000000000000000000000000000000000000000000000000000000000000000000000000000000000000000000000000B002000000000000008CFE1F
:3C0D9800000000000000000000000000000000000000000000000000000000000000000000000000000000000000000000000000000002000000000000003CFEE3
:3C0DD40000000000000000000000000000000000000000000000000000000000000000000000000000000000000000000000000000800600000000000000F8FE67
:3C0E100002000000000000000000000000000000000000000000000000000000000000000000000000000000000000000000000000805600000000000000DDFEF3
:3C0E4C0002000000000000000000000000000000000000000000000000000000000000000000000000000000000000000000000000800000000000000000AFFF3A
:3C0E8800000000000000000000000000000000000000000000000000000000000000000000000000000000000000000000000000000000000000000000001EFE12
:3C0EC40002000000000000000000000000000000000000000000000000000000000000000000000000000000000000000000000000800400000000000000EBFF82
:3C0F00000200000000000000000000000000000000000000000000000000000000800180010000000000000000000000000000000000120800000080010085FE93
:3C0F3C0000000000000000000000000000000000000000000000000000000000000000800600000000000000000000000000000000D002000000000000000AFE19
:3C0F7800000000000000000000000000000000000000000000000000000000000000000006000000000000000000000000000000000002000000000000005AFEDD
:3C0FB40000000000000000000000000000000000000000000000000000000000000000000000000000000000000000000000000000800600000000000000F8FE85
:3C0FF000020000000000000000000000000000000000000000000000000000000000008010020000000000000000000000000000008056000000000000006DFFEF
:3C102C000200000000000000000000000000000000000000000000000000000000000000000000000000000000000000000000000080080000000000000027FFD8
:3C106800000000000000000000000000000000000000000000000000000000000000000000000000000000000000000000000000000000000000000000001EFE30
:3C10A400020000000000000000000000000000000000000000000000000000000000008006000000000000000000000000000000008004000000000000000DFFF8
:3C10E0000200000000000000000000000000000000000000000000000000000000000000060000000000000000000000000000000000028201000080010053FF74
:3C111C00000000000000000000000000000000000000000000A8000000000000000000A2000000000000000000000000000000000090020000000000000024FE99
:3C11580000000000000000000000000000000000000000000000000000000000000000800000000000000000000000000000000000000200000000000000BCFE1F
:3C11940000000000000000000000000000000000000000000000000000000000000000000000000000000000000000000000000000800600000000000000F8FEA3
:3C11D00002000000000000000000000000000000000000000080000000000000000000801002000000000000000000000000000000C08E0000000000000031FE52
:3C120C00020000000000000000000000000000000000000000020000000000000000000000000000000000000000000000000000008010000000000000009FFE75
:3C1248000000000000000000000000000000000000000000000006000000000000000000000000000000000000000000000000000000000000000000000018FE4E
:3C1284000200000000000000000000000000000000000000008000000000000000000080060000000000000000000000000000000080040000000000000085FF1E
:3C12C000028001000000000000000000000000000000000000A007800180010000000080060000000000000000000000000000000000820000000000000047FE79
:3C12FC000000000000000000000000000000000000000000008206000000000000000088000000000000000000000000000000000088020000000000000092FE8C
:3C13380000000000000000000000000000000000000000000000060000000000000000000080000000000000000000000000000000000200000000000000B2FE41
:3C13740000000000000000000000000000000000000000000000060000000000000000000000000000000000000000000000000000800600000000000000FEFEB5
:3C13B000020000000000000000000000000000000000000000A0060000000000000000A01002000000000000000000000000000000C08E0000000000000035FE26
:3C13EC000200000000000000000000000000000000000000000000000000000000000000000000000000000000000000000000000080080000000000000027FF15
:3C142800008000800080008000800080008000800080008000800080008000800080008000800080008000800080008000800080008000800080008000009EFEEC
:3C146400020000000000000000000000000000000000000000000000000000000000000006000000000000000000000000000000000004000000010001001DFE23
:3C14A000020000000000008001000080010000000000000000800180018001800100008007800000000000800100000000000000000082000080008000007BFF84
:3C14DC00000000000000000000000000000000000000000000000000000000000000000004000000000000000000000000000000000000000000000000005AFE78
:3C1518000000000000000000000001800080008000000000010000000000000000000000008000800000008000000000000000000020000000000000000026FE51
:3C155400000000000000000000000000000000000000000000000000000000000000000000000000000000000000000000000000000000000000000000001EFE3F
:3C159000200000000000000000000000000000000000000000000000000000000000000000000000000000000000000000000000000000000000000000003CFEC5
:3C15CC00000000000000000000000000000000000000000000000000000000000000000000000000000000000000000000000000000000000000000000001EFEC7
:3C1608000000000000000000000000000000000000000000000000000000000000000000000000000000000000000000000000000000000000000000008096FE92
:3C16440000000000000000000000000000000000002000000000000000800000000000400000010000000000000000000000000000000000000000000000CCFFBE
:3C168000000000000000000001000000000000000000000040000000000000000000000000000000000000080000000000000000000000000100000000008AFE5C
:3C16BC000000000000000000000000000004000000000000000000000000000000000000000400000000000400000000000000000000002020000200010038FF6C
:3C16F8000000000000000000020000000000000000000002000000000000042000000002000002000000000000000000000000000000000000000000000049FF42
:3C1734000000001000000000000000800000000000000000000200000001000000000100000200020000000000000000000000000100040000000000002042FE7C
:3C17700000080000000000000000000000000000000000000000000000000000000000000000000000000000000000000000000000000100000000A00000B6FFDF
:3C17AC0000000000000000000000000000000000000000000000000000000000000000000000000000000000000000000000000000000200000000000008BCFE3D
:3C17E800002000000000000000000000040000000000000000002400000000000000000002000000000000000401000000000000000021100000000000007EFFC8
:3C182400004000000000000000000000000000000000000000000000020004000000000004000000000000000000000000200000408200040000000004009EFEB8
:3C1860002000220020000000000000000000000000000000000002000400000004000000000000000000000000000000000000000028100000000000000053FE57
:3C189C00000000000000000000000000000000000000000000000000000000000000000000000000000000000000000000000000000000000000000000001EFEF4
:3C18D800000000000000000000000000000000000000000000000000000000000000000000000000000000000000000000000000000000000000000000001EFEB8
:3C191400000000000000000000000000000000000000000000000000000000000000000000000000000000000000000000000000000000000000000000001EFE7B
:3C195000008000000000000000000002000000000000000000000000000000000000000000000002000000000000000000000000000000010000000000008EFE4A
:3C198C0000000000000000000008000000000000000000000000000000000000000000000000000000000000000000000000000000000000000000000020BCFE3D
:3C19C80000000000000000000000000000000000000000000080000000000000000040000000000000000000000000000000000000000000000000000000D2FE53
:3C1A040000000000200000100000000000000000800000000000000000000000000000100000001000000000000008000000000800004000000000000000A2FFE5
:3C1A40000000000000000000000000000000000000000000000000000000000000000000400000000000000000020000000000000000000000000000000038FEF2
:3C1A7C00000000000000000000000000000000000000000000000000000000000000000000000000000000000000000000000000000000000000000000001EFE12
:3C1AB80000000000000000000000000000000000000000000000000000000000000000000000000000000000000000000000000400010000080000000800CAFF14
:3C1AF400000000008000000000000008000000000000000010000000000000000000000000000000000000000000000000000000000010080000000800009EFE62
:3C1B30008000000000000000000000000000000000000000000000000000000000000000000000000000000000000000000000000000000000000000000096FE65
:3C1B6C0000000000000000000000000000000000000000000000000000000000000000100000000000000000000000000000000000100000010001000580D2FEC6
:3C1BA800000000000000000000000000000000000000000000000000000000000000000000000000000000000000000000000000000000000000000000001EFEE5
:3C1BE4000000000000000000000000000000000000000000000000000000000000000000000100000000000000000000000000200004000800000002800082FE96
:3C1C2000000000000000000000000004000000000004000400100004000400040000004000000000000000000000000000000000000100000000000000004AFED7
:3C1C5C004000010000000000000000000000000000000000000000000000000000000004000000000040004000400040004000400000400000000010200048FFD0
:3C1C98000800000000000000000020000000000000000000000400000000000000000000000000000002000000000000000000000000080000000000000074FE68
:3C1CD40008000000000000000000000000000000000000080000000000000000000000000000000000000000000000000000000000200000000000000000B6FEF0
:3C1D1000000000000000000000000000000000020000000000000000000000000000000002000000000000000000000000000000000000000000000000001CFE79
:3C1D4C00000000000000000000000000000000000000000000000000000000000000000000000000000000000000000000000000000000000000000000000FFF4D
:3C1D8800000000000000000000000000000000000000000000000000000000000000000000000000000000000000000000000000000000000000000000001EFE03
:3C1DC400000000000000000000000000000000000000000000000000000000000000000000000000000000000000000000000000000000000000000000001EFEC7
:3C1E0000020000000000000000000000000000000000000000000000000000000000000000000000000000000000000000000000000000000000000000003EFE68
:3C1E3C00020000000000000000000000000000000000000000000000000000000000000000000000000000000000000000000000000000000000000000002FFF3A
:3C1E7800000000000000000000000000000000000000000000000000000000000000000000000000000000000000000000000000000000000000000000000FFF20
:3C1EB400020000000000000000000000000000000000000000000000000000000000000000000000000000000000000000000000000000000000000000003EFEB4
:3C1EF000020000000000000000000000000000000000000000000000000000000000000000000000000000000000000000000000000000000000000000003EFE78
:3C1F2C00020000000000000000000000000000000000000000000000000000000000000000000000000000000000000000000000000000000000000000003EFE3B
:3C1F6800000000000000000000000000000000000000000000000000000000000000000000000000000000000000000000000000000000000000000000001EFE21
:3C1FA400000000000000000000000000000000000000000000000000000000000000000000000000000000000000000000000000000000000000000000001EFEE5
:3C1FE000020000000000000000000000000000000000000000000000000000000000000000000000000000000000000000000000000000000000000000002FFF95
:3C201C00020000000000000000000000000000000000000000000000000000000000000000000000000000000000000000000000000000000000000000002FFF58
:3C205800020000000000000000000000000000000000000000000000000000000000000000000000000000000000000000000000000000000000000000002FFF1C
:3C209400020000000000000000000000000000000000000000000000000000000000000000000000000000000000000000000000000000000000000000003EFED2
:3C20D0000A080000000000000000000000000000000000000000000000000000000000000000000000000000000000000000000000000000000000000000B6FE0E
:3C210C00000000000000000000000000000000000000000000000000000000000000000000000000000000000000000000000000000000000000000000001EFE7B
:3C214800000000000000000000000000000000000000000000000000000000000000000000000000000000000000000000000000000000000000000000001EFE3F
:3C218400000000000000000000000000000000000000000000000000000000000000000000000000000000000000000000000000000000000000000000001EFE03
:3C21C000020000000000000000000000000000000000000000000000000000000000000000000000000000000000000000000000000000000000000000002FFFB3
:3C21FC00020000000000000000000000000000000000000000000000000000000000000000000000000000000000000000000000000000000000000000002FFF77
:3C223800000000000000000000000000000000000000000000000000000000000000000000000000000000000000000000000000000000000000000000001EFE4E
:3C227400020000000000000000000000000000000000000000000000000000000000000000000000000000000000000000000000000000000000000000002FFFFE
:3C22B000020000000000000000000000000000000000000000000000000000000000000000000000000000000000000000000000000000000000000000002FFFC2
:3C22EC00020000000000000000000000000000000000000000000000000000000000000000000000000000000000000000000000000000000000000000003EFE78
:3C232800000000000000000000000000000000000000000000000000000000000000000000000000000000000000000000000000000000000000000000001EFE5D
:3C236400000000000000000000000000000000000000000000000000000000000000000000000000000000000000000000000000000000000000000000001EFE21
:3C23A000000000000000000000000000000000000000000000000000000000000000000000000000000000000000000000000000000000000000000000000FFFF3
:3C23DC00020000000000000000000000000000000000000000000000000000000000000000000000000000000000000000000000000000000000000000002FFF95
:3C241800020000000000000000000000000000000000000000000000000000000000000000000000000000000000000000000000000000000000000000003EFE4A
:3C245400020000000000000000000000000000000000000000000000000000000000000000000000000000000000000000000000000000000000000000002FFF1C
:3C2490000A100000000000000000000000000000000000000000000000000000008001000000000000000000000000000000000000000000000000000000A7FFCF
:3C24CC0000000000000000000000000000000000000000000000000000A10600000000000000000000000000000000000000000000000000000000000000D9FE56
:3C250800000000000000000000000000000000000000000000000000000000000000000000000000000000000000000000000000000000000000000000001EFE7B
:3C25440000000000000000000000000000000000000000000000000000800600000000000000000000000000000000000000000000000000000000000000F8FEDF
:3C25800002000000000000000000000000000000000000000000000000803000000000000000000000000000000000000000000000000000000000000000ACFFC2
:3C25BC0002000000000000000000000000000000000000000000000000810000000000000000000000000000000000000000000000000000000000000000BFFEA3
:3C25F800000000000000000000000000000000000000000000000000000000000000000000000000000000000000000000000000000000000000000000000FFF99
:3C26340002000000000000000000000000000000000000000000000000800600000000000100000000000000000000000000000000000000000000000000D8FF0A
:3C2670000200000000000000000000000000000000000000000000000040060000000080000000000000000000000000000000000000000000000000000098FED0
:3C26AC00000000000000000000000000000000000000000000000000000000000000000000000000000000000000000000000000000000000000000000001EFED6
:3C26E800000000000000000000000000000000000000000000000000000000000000000000000000000000000000000000000000000000000000000000001EFE9A
:3C272400000000000000000000000000000000000000000000000000000000000000000000000000000000000000000000000000000000000000000000001EFE5D
:3C276000020000000000000000000000000000000000000000000000000000000000000000000000000000000000000000000000000000000000000000002FFF0D
:3C279C00020000000000000000000000000000000000000000000000000000000000000000000000000000000000000000000000000000000000000000002FFFD1
:3C27D800000000000000000000000000000000000000000000000000000000000000000000000000000000000000000000000000000000000000000000001EFEA9
:3C281400020000000000000000000000000000000000000000000000000000000000000000000000000000000000000000000000000000000000000000002FFF58
:3C285000020000000000000000000000000000000000000000000000000000000000000000000000000000000000000000000000000000000000000000002FFF1C
:3C288C00000000000000000000000000000000000000000000000000000000000000000000000000000000000000000000000000000000000000000000000FFF02
:3C28C800000000000000000000000000000000000000000000000000000000000000000000000000000000000000000000000000000000000000000000001EFEB8
:3C290400000000000000000000000000000000000000000000000000000000000000000000000000000000000000000000000000000000000000000000001EFE7B
:3C294000020000000000000000000000000000000000000000000000000000000000000000000000000000000000000000000000000000000000000000003EFE1D
:3C297C00020000000000000000000000000000000000000000000000000000000000000000000000000000000000000000000000000000000000000000002FFFEF
:3C29B800000000000000000000000000000000000000000000000000000000000000000000000000000000000000000000000000000000000000000000000FFFD5
:3C29F400020000000000000000000000000000000000000000000000000000000000000000000000000000000000000000000000000000000000000000003EFE69
:3C2A300002000000000000000080010000000000000000000000000000000000000000000000000000000000000000000000000000000000000000000000A6FF42
:3C2A6C00000000000000000000000000000000000000000000000000000000000000000000000000000000000000000000000000000000000000000000000FFF20
:3C2AA800000000000000000000000000000000000000000000000000000000000000000000000000000000000000000000000000000000000000000000001EFED6
:3C2AE400000000000000000000000000000000000000000000000000000000000000000000000000000000000000000000000000000000000000000000001EFE9A
:3C2B2000020000000000000000000000000000000000000000000000000000000000000000000000000000000000000000000000000000000000000000003EFE3B
:3C2B5C00020000000000000000000000000000000000000000000000000000000000000000000000000000000000000000000000000000000000000000002FFF0D
:3C2B9800000000000000000000000000000000000000000000000000000000000000000000000000000000000000000000000000000000000000000000000FFFF3
:3C2BD400020000000000000000000000000000000000000000000000000000000000000000000000000000000000000000000000000000000000000000003EFE87
:3C2C1000020000000000000000000000000000000000000000000000000000000000000000000000000000000000000000000000000000000000000000003EFE4A
:3C2C4C00088206000000000000000000000000000000000000000000000000000000000000000000000000000000000000000000000000000000000000007AFE44
:3C2C88000000060000000000000000000000000000000000000000000000000000000000000000000000000000000000000000000000000000000000000078FE94
:3C2CC4000000060000000000000000000000000000000000000000000000000000000000000000000000000000000000000000000000000000000000000078FE58
:3C2D000002A40600000000000000000000000000000000000000000000000000000000000000000000000000000000000000000000000000000000000000EDFFFF
:3C2D3C00020000000000000000000000000000000000000000000000000000000000000000000000000000000000000000000000000000000000000000002FFF2B
:3C2D7800020000000000000000000000000000000000000000000000000000000000000000000000000000000000000000000000000000000000000000003EFEE1
:3C2DB40002800000000000000000000000000000000000000000000000000000000000000000000000000000000000000000000000000000000000000000AFFFB3
:3C2DF000080400000000000000000000000000000000000000000000000000000000000000000000000000000000000000000000000000000000000000008BFF11
:3C2E2C0000C20000000000000000000000000000000000000000000000000000000000000000000000000000000000000000000000000000000000000000CDFFDC
:3C2E6800000000000000000000000000000000000000000000000000000000000000000000000000000000000000000000000000000000000000000000001EFE12
:3C2EA400000000000000000000000000000000000000000000000000000000000000000000000000000000000000000000000000000000000000000000001EFED6
:3C2EE00002800000000000000000000000000000000000000000000000000000000000000000000000000000000000000000000000000000000000000000BEFE78
:3C2F1C00020200000000000000000000000000000000000000000000000000000000000000000000000000000000000000000000000000000000000000002DFF49
:3C2F580000800680008000800080008000800080008000800080008000800080008000800080008000800080008000800080008000800080008000800000E9FF4F
:3C2F9400020000000000000000000000000000000000000000000000000000000000000000000000000000000000000000000000000000000000000000003EFEC3
:3C2FD00002A0070000000000000000000000000000000000000000000000008001000000000000000000000000000000000000000000000000000000000060FE3D
:3C300C00000000000000000000000000000000000000000000000000000000000000000000000000000000000000000000000000000000000000000000001EFE6C
:3C30480000000080000000000000000000000000000000000000000000200000000000000000000000000000000000000000000000000000000000000000B6FEF8
:3C308400000000000000000000000000000000000000000000000000000000000000000000000000000000000000000000000000000000000000000000001EFEF4
:3C30C000000000000000000000000000000000000000000000000000000000000000000000000000000000000000000000000000000000000000000000001EFEB8
:3C30FC00000000000000000000000000000000000000000000000000000000000000000000000000000000000000000000000000000000000000000000001EFE7C
:3C313800000000000000000000000000000000000000000000000000000000000000000000000000000000000000000000000000000000000000000000001EFE3F
:3C317400000000000000000000000000000000000000000000000000000000000000000000000000000000000000000000000000000000000000000000001EFE03
:3C31B000000000000000000000000000000000000000000000000000000000000000000000000000000000000000000000000000000000000000000000001EFEC7
:3C31EC00000000000000000000000000000000000000000000000000000000000000000000000000000000000000000000000000000000000000000000001EFE8B
:3C322800020400000000000000000000000000000000000000000000000000000000000001000000000000000000000000000000000000000000000000003AFF2A
:3C326400000200000000000000000000000000000000000000000000000000000000010000000000000000000000000000000000000000000000000000000CFE21
:3C32A000001000000000000000000000000000000000000000000000000004000000000000000000000000000000000000000000000000000000000000004AFE96
:3C32DC00000000000000000000000000000000000000000000000000000000000000000000000000000000000000000000000000000000000000000000001EFE9A
:3C331800000000000000000000000000000000000000000000000000400000000400000000000000000000000000000000000000000000000000000000005EFED9
:3C335400000000000000000000000000000000000000000000000000000000000000000000000000000000000000000000000000000000000000000000001EFE21
:3C339000001004000000000000000000000000000000000000000000000000000000000000000000000000000000000000000000000000000000000000004AFEA5
:3C33CC00000000000000000000000000000000000000000000000000000000000000000000000000000000000000000000000000000000000000000000001EFEA9
:3C340800000000000000000000000000000000000000000000000000000000000000000000000000000000000000000000000000000000000000000000001EFE6C
:3C344400000000000000000000000000000000000000000000000000000000000000000000000000000000000000000000000000000000000000000000001EFE30
:3C348000000200000000000000000000000000000000000000000000000000000000000000000000000000000000000000000000000000000000000000001CFEF4
:3C34BC00000000000000000000000000000000000000000000000000000000000000000000000000000000000000000000000000000000000000000000001EFEB8
:3C34F800000000000000000000000000000000000000000000000000000000000000000000000000000000000000000000000000000000000000000000001EFE7C
:3C353400000000000000000000000000000000000000000000000000000000000000000000000000000000000000000000000000000000000000000000001EFE3F
:3C357000000000000000000000004000000000000000000000000000000100000000000000000000000000000000000000000000000000000000000000004EFF91
:3C35AC00000000000000000000000000000000000000000000000000000000000000000000000000000000000000000000000000000000000000000000001EFEC7
:3C35E800000000000000000000000000000000000000000000000000000000000000000000000000000000000000000000000000000000000000000000001EFE8B
:3C362400000000000000000000000000000000000000000000000000000000000000000000000000000000000000000000000000000000000000000000001EFE4E
:3C366000000000000000000000000000000000000000000000000000000000000000000000000000000000000000000000000000000000000000000000001EFE12
:3C369C00000000000000000000000000000000000000000000000000000000000000000000000000000000000000000000000000000000000000000000001EFED6
:3C36D800000000000000000000000000000000000000000000000000000000000000000000000000000000000000000000000000000000000000000000001EFE9A
:3C371400000000000000000000000000000000000000000000000000000000000000000000000000000000000000000000000000000000000000000000001EFE5D
:3C375000000000000000000000000000000000000000000000000000000000000000000000000000000000000000000000000000000000000000000000001EFE21
:3C378C00000000000000000000000000000000000000000000000000000000000000000000000000000000000000000000000000000000000000000000001EFEE5
:3C37C800000000000000000000000000000000000000000000000000000000000000000000000000000000000000000000000000000000000000000000001EFEA9
:3C380400000000000000000000000000000000000000000000000000000000000000000000000000000000000000000000000000000000000000000000001EFE6C
:3C384000000000020000000000000000000000000000000000000000000000000000000000000000000000000000000000000000000000000000000000003EFE0E
:3C387C00000000000000000000000000000000000000000000000000000000000000000000000000000000000000000000000000000000000000000000001EFEF4
:3C38B800000000000000000000000000000000000000000000000000000000000000000000000000000000000000000000000000000000000000000000001EFEB8
:3C38F400000000000000000000000000000000000000000000000000000000000000000000000000000000000000000000000000000000000000000000001EFE7C
:3C393000020000000000000000000000000000000000000000000000000000000000000000000000000000000000000000000000000000000000000000002FFF2B
:3C396C00020000000000000000000000000000000000000000000000000000000000000000000000000000000000000000000000000000000000000000002FFFEF
:3C39A800000000000000000000000000000000000000000000000000000000000000000000000000000000000000000000000000000000000000000000001EFEC7
:3C39E400020000000000000000000000000000000000000000000000000000000000000000000000000000000000000000000000000000000000000000002FFF77
:3C3A2000020000000000000000000000000000000000000000000000000000000000000000000000000000000000000000000000000000000000000000002FFF3A
:3C3A5C000800000000000000000000C206000000000000000000000000000000000000000000000000000000000000000000000000000000000000000000D0FE90
:3C3A9800000000000000000000000000060000000000000000000000000000000000000000000000000000000000000000000000000000000000000000007EFE70
:3C3AD4000000000000000000000000800200000000000000000000000000000000000000000000000000000000000000000000000000000000000000000036FE00
:3C3B10000204000000000000000000801202000000000000000000000000000000000000000000000000000000000000000000000000000000000000000001FEE0
:3C3B4C001200000000000000000000800400000000000000000000000000000000000000000000000000000000000000000000000000000000000000000067FE42
:3C3B8800020000000000000000000000020000000000000000000000000000000000000000000000000000000000000000000000000000000000000000001EFEE1
:3C3BC4000200000000000000000000800000000000000000000000000000000000000000000000000000000000000000000000000000000000000000000027FF1D
:3C3C000000020000000000000000000028000000000000000000000000000000000000000000008001000000000000000000000000000000000000000000B7FF27
:3C3C3C000800000000000088060080C0060000000000000000000000000000000000000000000000000000000000000000000000000000000000000000008DFFE4
:3C3C78000000000000000000060000000600000000000000000000000000000000000000000000000000000000000000000000000000000000000000000018FEEE
:3C3CB4000000000000000080020000800200000000000000000000000000000000000000000000000000000000000000000000000000000000000000000094FE3E
:3C3CF00002040000000000A01202008012020000000000000000000000000000000000000000000000000000000000000000000000000000000000000000B3FF98
:3C3D2C0002000000000000800C0000800C000000000000000000000000000000000000000000000000000000000000000000000000000000000000000000ABFF97
:3C3D6800020000000000000002000000020000000000000000000000000000000000000000000000000000000000000000000000000000000000000000002DFFED
:3C3DA40002000000000000800000008000000000000000000000000000000000000000000000000000000000000000000000000000000000000000000000A7FF3B
:3C3DE0008800000000000000200000002000000000000000000000000000000000000000000000000000000000000000000000000000000000000000000027FFB9
:3C3E1C0008000000000000A8060000C2060000000000000000000000000000000000000000000000000000000000000000000000000000000000000000000FFFDE
:3C3E58000000000000000000060000000600000000000000000000000000000000000000000000000000000000000000000000000000000000000000000018FE0C
:3C3E94000000000000000080020000800200000000000000000000000000000000000000000000000000000000000000000000000000000000000000000094FE5C
:3C3ED00002040000000000800A0100800A010000000000000000000000000000000000000000000000000000000000000000000000000000000000000000A9FEF3
:3C3F0C0012000000000000801400008014000000000000000000000000000000000000000000000000000000000000000000000000000000000000000000B3FE8E
:3C3F4800020000000000000002000000020000000000000000000000000000000000000000000000000000000000000000000000000000000000000000002DFF0B
:3C3F840002000000000000800000008000000000000000000000000000000000000000000000000000000000000000000000000000000000000000000000A7FF59
:3C3FC00000080000000000002080010020000000000000000000000000000000000000000000000000000000000000000000000000000000000000000000BFFE3F
:3C3FFC000800000000000084060080C00600000000000000000000000000000000000000000000000000000000000000000000000000000000000000000081FF31
:3C4038000000000000000000060000000600000000000000000000000000000000000000000000000000000000000000000000000000000000000000000018FE2A
:3C4074000000000000000080020000800200000000000000000000000000000000000000000000000000000000000000000000000000000000000000000094FE7A
:3C40B00002040000000000C00A0100800A010000000000000000000000000000000000000000000000000000000000000000000000000000000000000000E9FE91
:3C40EC0002000000000000800400008004000000000000000000000000000000000000000000000000000000000000000000000000000000000000000000A3FFEC
:3C412800020000000000000002000000020000000000000000000000000000000000000000000000000000000000000000000000000000000000000000002DFF29
:3C41640002000000000000800000008000000000000000000000000000000000000000000000000000000000000000000000000000000000000000000000A7FF77
:3C41A00090000000000000003000000030000000000000000000000000000000000000000000000000000000000000000000000000000000000000000000B7FE3E
:3C41DC00080000000000000000000000000000000000000000000000000000000000000000000000000000000000000000000000000000000000000000008FFF11
:3C421800000000000000000000000000000000000000000000000000000000000000000000000000000000000000000000000000000000000000000000001EFE4E
:3C425400000000000000000000000000000000000000000000000000000000000000000000000000000000000000000000000000000000000000000000001EFE12
:3C429000020400000000000000000000000000000000000000000000000000000000000000000000000000000000000000000000000000000000000000002BFFC2
:3C42CC000A000000000000000000000000000000000000000000000000000000000000000000000000000000000000000000000000000000000000000000AFFFFE
:3C430800020000000000000000000000000000000000000000000000000000000000000000000000000000000000000000000000000000000000000000002FFF49
:3C434400020000000000000000000000000000000000000000000000000000000000000000000000000000000000000000000000000000000000000000002FFF0D
:3C438000000200000000000000000000000000000000000000000000000000000000000000000000000000000000000000000000000000000000000000000DFFF3
:3C43BC0000000000000000000000000000000000000000000000000000000000000000000000000000000000000000000000000000000000000000821600EAFF44
:3C43F8000000000000000000000000000000000000000000000000000000000000000000000000000000000000000000000000000000000000000000060078FE0D
:3C44340000000000000000000000000000000000000000000000000000000000000000000000000000000000000000000000000000000000000000800200BCFE10
:3C44700002000000000000000000000000000000000000000000000000000000000000000000000000000000000000000000000000000000000000C00210CDFE71
:3C44AC0002000000000000000000000000000000000000000000000000000000000000000000000000000000000000000000000000000000000000800000AFFFA4
:3C44E800000000000000000000000000000000000000000000000000000000000000000000000000000000000000000000000000000000000000000000001EFE7C
:3C452400020000000000000000000000000000000000000000000000000000000000000000000000000000000000000000000000000000000000008002008DFF4B
:3C45600002000000000000000080010000000000000000000000000000000000000000000000000000000000000000000000000000000000000000001404A3FFE2
:3C459C0008000000000000D0060000D006000000000000000000000000000000000000000000000000000000000000000000000000000000000000D00200B7FEA8
:3C45D800000000000000000000000000000000000000000000000000000000000000000000000000000000000000000000000000000000000000000002003CFE6B
:3C4614000000000000000080060000800600000000000000000000000000000000000000000000000000000000000000000000000000000000000080060076FE64
:3C4650000204000000000080160200801602000000000000000000000000000000000000000000000000000000000000000000000000000000000080160430FF2F
:3C468C000A000000000000A80000008200000000000000000000000000000000000000000000000000000000000000000000000000000000000000801000BDFE73
:3C46C800020000000000000000000000000000000000000000000000000000000000000000000000000000000000000000000000000000000000000000002FFF86
:3C4704000200000000000080000000800000000000000000000000000000000000000000000000000000000000000000000000000000000000000080040072FE83
:3C47400000080000000000000600004006000000000000000000008001000000000000000000000000000000000000000000000000000000000000000208AEFEB2
:3C477C0008000000000000900600009006000000000000000000000000000000000000000000000000000000000000000000000000000000000000900600F7FE42
:3C47B800000000000000000000000000000000000000000000000000000000000000000000000000000000000000000000000000000000000000000000001EFEA9
:3C47F4000000000000000080060000800600000000000000000000000000000000000000000000000000000000000000000000000000000000000080060076FE83
:3C48300002040000000000C0160200C016020000000000000000000000000000000000000000000000000000000000000000000000000000000000C0160434FF89
:3C486C000200000000000084000000C100000000000000000000000000000000000000000000000000000000000000000000000000000000000080C00000EFFE9C
:3C48A800020000000000000000000000000000000000000000000000000000000000000000000000000000000000000000000000000000000000000000002FFFA4
:3C48E4000200000000000080000000800000000000000000000000000000000000000000000000000000000000000000000000000000000000000080000027FFF0
:3C492000100800000000004006000000060000000000000000800180010000000000000000000000000000800100000000000000000000000000000006003FFE31
:3C495C0002000000000000880600008806000000000000000000000000000000000000000000000000000000000000000000000000000000000000880600CFFFA5
:3C4998000000000000000000000000000000000000000000000000000000000000000000000000000000000000000000000000000000000000000000060078FE67
:3C49D4000000000000000080060000800600000000000000000000000000000000000000000000000000000000000000000000000000000000000080020032FEE9
:3C4A100000000000000000C00E0100C00E010000000000000000000000000000000000000000000000000000000000000000000000000000000000A00A0856FFC5
:3C4A4C000000000000000088000000C1000000000000000000000000000000000000000000000000000000000000000000000000000000000000008000001AFF4C
:3C4A8800008000800080008000800080008000800080008000800080008000800080008000800080008000800080008000800080008000800080008000009EFE56
:3C4AC400000000000000000000000000000000000000000000000000000000000000000000000000000000000000000000000000000000000000000002003CFE7A
:3C4B000000800100000000200600000006000000000000000000000000000000000000000080018001000080010000000000000000000000000000001404B4FE7F
:3C4B3C00000000000000000000000000000000000000000000000000000000000000000000000000000000000000000000000000000000000000000000001EFE21
:3C4B780000000080008000200080002000800000008000000000000000000000000000000000000000000000000000000000000000000080000000A0000094FE8F
:3C4BB400000000000000000000000000000000000000000000000000000000000000000000000000000000000000000000000000000000000000000002003CFE89
:3C4BF000200000000000000000000000000000000000000000000000000000000000000000000000000000000000000000000000000000000000000000003CFE2F
:3C4C2C00000000000000000000000000000000000000000000000000000000000000000000000000000000000000000000000000000000000000000000001EFE30
:3C4C6800000000000000000000000000000000000000000000000000000000000000000000000000000000000000000000000000000000000000000000001EFEF4
:3C4CA400000000000000000000000000000000000000000000000000000000000000000000000000000000000000000000000000000000000000000000001EFEB8
:3C4CE000000000000000000000000000000000000000000000000000000000000000000000000000000000000000000000000000000000000000000000001EFE7C
:3C4D1C0080000000000000002000010020000000000000000000000000000000000000000000000000000000000000000000000000000000000000000000A6FFF5
:3C4D580002000000000000000000000000000000000000000000000000000000000000000000000000000000000000000000000000000000000000800000BEFEE1
:3C4D9400000000000000000000000000000000000000000000000000000000000000000000000000000000000000000000000000000000000000000000001EFEC7
:3C4DD000000000000000000000000000000000000000000000000000000000000000000000000000000000000000000000000000000000000000000000001EFE8B
:3C4E0C00040000000000000000000000000000000000000000000000000000000000000000000000000000000000000000000000000000000000000000005EFE0A
:3C4E4800000000000000000000002001000000000000000000000200020000000000000000000000000000000000000000000000000000000000000000001CFFEE
:3C4E840000000000000000400000000C00000000000000000000000000000000000000000000040004000000020000000000000000000000000020480000BEFE78
:3C4EC0000010040000000008000000000000000000000000000000000000000000000000000000000000000004000000000000000000000000000000000046FE52
:3C4EFC00000000000000000000000000000000000000000000000000000000000000000000000000000000000000000000000000000000000000000000001EFE5E
:3C4F3800000000000000000000000000000000000000000000000000000000000000000000000010000000000000000000000000000000000000000000202CFFE2
:3C4F7400000400000000000000000000080000000000000000000000000000000000000000000000000000000000000000000000000000000000000000009AFE5D
:3C4FB000000000020000000000000000000000000000000000000000000000000000000000000000000000000000000000000000000000020000000200001CFEA5
:3C4FEC00000000000000000000000000000000000000000000000000000000000000000000000000000000000000000000000000000000000000000000001EFE6D
:3C502800000000000000000000000000000000000000000000000000000000000000000000000000000000000000000000000000000000000000000000001EFE30
:3C506400000000000000000000000000000000000000000000000000000000000000000000000000000000000000000000000000000000000000000000001EFEF4
:3C50A000000000000000000000024000000200000000000000000000000000000000000000000000000000000000000000000000000000000000000000007CFE16
:3C50DC00000000000000000000000000000000000000000000000000000000000000000000000000000000000000000000000000000000000000000000001EFE7C
:3C511800000000000000000000000000000000000000000000000000000000000000000000000000000000000000000000000000000000000000000000001EFE3F
:3C515400000000000000000000000000000000000000000000000000000000000000000000000000000000000000000000000000000000000000000000001EFE03
:3C519000000000000000000000000000000000000000000000000000000000000000000000000000000000000000000000000000000000000000000000001EFEC7
:3C51CC00200000000000000000000010000000000000000000000000000000000000000000000000000000000000000000000000000000000000000000002CFF4C
:3C52080000800100000000500000000000000000000000000000000000000000000000000000000000000000000000000000000000000000000000000000CEFFCC
:3C524400000000000000000000000000000000000000000000000000000000000000000000000000000000000000000000000000000000000000000000001EFE12
:3C528000002000000000008000000040000000000000000000000000080000000000000000000000000000000000000000000000000000000000000000002BFFE0
:3C52BC00500000000000000000000000400000000000000000000000000000000000000000000000000000000000000000000000000000000000000000001EFF09
:3C52F8001002000000000000080000000000000000000000000000000000000000000000000000000000000000000000000000000000000000000000000094FFCD
:3C53340008000000000000000600000006000000000000000000000000000000000000000000000000000000000000000000000000000000000000280000B0FE53
:3C537000000000000002000200020002000200000002000000000000000000000000000000000000000000000000000000000000000000000000000000001CFEDB
:3C53AC0000000000000000000000000000000000000000000000000000000000000000000000000000000000000000000000000000000000000000B0080037FFD7
:3C53E800000000000000000000000000000000000000000000000000000000000000000000000000000000000000000000000000000000000000000000001EFE6D
:3C542400000000000000000000000000000000000000000000000000000000000000000000000000000000000000000000000000000000000000000000001EFE30
:3C54600002000000000000000000000000000000000000000000000000000000000000000000000000000000000000000000000000000000000000808400F2FE1A
:3C549C00020000000000000000000000000000000000000000000000000000000000000000000000000000000000000000000000000000000000000100003FFE94
:3C54D800000000000000000000000000000000000000000000000000000000000000000000000000000000000000000000000000000000000000000000000FFF8A
:3C55140002000000000000000000000000000000000000000000000000000000000000000000000000000000000000000000000000000000000000800000AFFF2B
:3C55500002000000000000000000000000000000000000000000000000000000000000000000000000000000000000000000000000000000000000401008FFFEC8
:3C558C00020000000000000000000000000000000000000000000000000000000000000000000000000000000000000000000000000000000000000000002FFFB3
:3C55C800000000000000000000000000000000000000000000000000000000000000000000000000000000000000000000000000000000000000000000001EFE8B
:3C560400000000000000000000000000000000000000000000000000000000000000000000000000000000000000000000000000000000000000000000001EFE4E
:3C564000020000000000000000000000000000000000000000000000000000000000000000000000000000000000000000000000000000000000000000003EFEF0
:3C567C00020000000000000000000000000000000000000000000000000000000000000000000000000000000000000000000000000000000000000000002FFFC2
:3C56B800020000000000000000000000000000000000000000000000000000000000000000000000000000000000000000000000000000000000000000002FFF86
:3C56F400020000000000000000000000000000000000000000000000000000000000000000000000000000000000000000000000000000000000000000003EFE3C
:3C5730000A080000000000000000000000000000000000000000000000000000000000000000000000000000000000000000000000000000000000000000B6FE77
:3C576C00000000000000000000000000000000000000000000000000000000000000000000000000000000000000000000000000000000000000000000001EFEE5
:3C57A800000000000000000000000000000000000000000000000000000000000000000000000000000000000000000000000000000000000000000000001EFEA9
:3C57E400000000000000000000000000000000000000000000000000000000000000000000000000000000000000000000000000000000000000000000001EFE6D
:3C582000020000000000000000000000000000000000000000000000000000000000000000000000000000000000000000000000000000000000000000002FFF1C
:3C585C00020000000000000000000000000000000000000000000000000000000000000000000000000000000000000000000000000000000000000000002FFFE0
:3C589800000000000000000000000000000000000000000000000000000000000000000000000000000000000000000000000000000000000000000000001EFEB8
:3C58D400020000000000000000000000000000000000000000000000000000000000000000000000000000000000000000000000000000000000000000002FFF68
:3C591000020000000000000000000000000000000000000000000000000000000000000000000000000000000000000000000000000000000000000000002FFF2B
:3C594C0002000000000000000000000000000000000000000000000000000000000000000000000000000000000000000000000000000084120000B00800CDFF03
:3C598800000000000000000000000000000000000000000000000000000000000000000000000000000000000000000000000000000000000200000000001CFEC7
:3C59C40000000000000000000000000000000000000000000000000000000000000000000000000000000000000000000000000000000080020000000400D0FE53
:3C5A0000000000000000000000000000000000000000000000000000000000000000000000000000000000000000000000000000000000A02200008080001EFE8C
:3C5A3C0002000000000000000000000000000000000000000000000000000000000000000000000000000000000000000000000000000080100000010000A7FEF6
:3C5A7800020000000000000000000000000000000000000000000000000000000000000000000000000000000000000000000000000000000000000000002FFFC2
:3C5AB4000200000000000000000000000000000000000000000000000000000000000000000000000100000001000100000000000000008006000080000020FF8C
:3C5AF0000A100000000000000000000000000000000000000000000000000000008001000000008000000080008000000000000000000000060400401008ACFF52
:3C5B2C0002000000000000000000000000000000000000000000000000000000000000C2060000000000000000000000000000810E0000A1060000000000CEFF70
:3C5B6800000000000000000000000000000000000000000000000000000000000000000000000000000000000000000000000000000000000000000000001EFEE5
:3C5BA4000000000000000000000000000000000000000000000000000000000000000080060000000000000000000000000000000000008006000000000076FE45
:3C5BE0000200000000000000000000000000000000000000000000000000000000000080300000000000000000000000000000C0400000803000000000004DFEDC
:3C5C1C0002000000000000000000000000000000000000000000000000000000000080A000000000000000000000000000000008000080A00000000000002DFFD6
:3C5C5800020000000000000000000000000000000000000000000000000000000000000000000000000000000000000000000000000000000000000000003EFED2
:3C5C9400020000000000000000000000000000000000000000000000000000000000008006000000010000000000000000000080000000800600000000005FFFE7
:3C5CD0000200000000000000000000000000000000000000000000000000000000000000060000800000000000000000000000200000000006000000000045FFA6
:3C5D0C0002000000000000000000000000000000000000000000000000000000000000000000000000000000000000000000000000000000000080A0000007FF33
:3C5D4800000000000000000000000000000000000000000000000000000000000000000000000000000000000000000000000000000000000000000000001EFE03
:3C5D8400000000000000000000000000000000000000000000000000000000000000000000000000000000000000000000000000000000000000000000001EFEC7
:3C5DC00002000000000000000000000000000000000000000000000000000000000000000000000000000000000000000000000000000000000000809000A6FFF0
:3C5DFC000200000000000000000000000000000000000000000000000000000000000000000000000000000000000000000000000000000000008000020085FF63
:3C5E3800020000000000000000000000000000000000000000000000000000000000000000000000000000000000000000000000000000000000000000002FFFFE
:3C5E740002000000000000000000000000000000000000000000000000000000000000000000000000000000000000000000000000000000000000800000BEFEB4
:3C5EB000020000000000000000000000000000000000000000000000000000000000000000000000000000000000000000000000000000000000002050000AFF3B
:3C5EEC0008000000000000000000000000000000000000000000000000000000000000000000000000000000000000000000000000000000000000A200002DFFA4
:3C5F2800000000000000000000000000000000000000000000000000000000000000000000000000000000000000000000000000000000000000000000001EFE21
:3C5F6400000000000000000000000000000000000000000000000000000000000000000000000000000000000000000000000000000000000000000000001EFEE5
:3C5FA00002080000000000000000000000000000000000000000000000000000000000000000000000000000000000000000000000000000000000801010A6FE77
:3C5FDC0012000000000000000000000000000000000000000000000000000000000000000000000000000000000000000000000000000000000080400000E7FED2
:3C601800020000000000000000000000000000000000000000000000000000000000000000000000000000000000000000000000000000000000000000002FFF1C
:3C60540002000000000000000000000000000000000000000000000000000000000000000000000000000000000000000000000000000000000000800600D8FEB2
:3C6090000008000000000080010000000000000000000000000000000000000000000000000000000000000000000000000000000000000000000000000096FFB6
:3C60CC00000000000000000000880800000000000000000000000000000000000000000000000088080000000000000000000000000000000000008200009CFE5C
:3C610800000000000000000000000000000000000000000000000000000000000000000000000000060000000000000000000000000000000000000000007EFED9
:3C614400000000000000000000000000000000000000000000000000000000000000000000000000000000000000000000000000000000000000000000001EFE03
:3C618000020000000000000000A040000000000000000000000000000000000000000000000000A040000000000000000000000000000000000000C010105BFFE7
:3C61BC00020000000000000000240000000000000000000000000000000000000000000000000001000000000000000000000000000000000000804008000DFEAD
:3C61F800000000000000000000000000000000000000000000000000000000000000000000000000000000000000000000000000000000000000000000001EFE4F
:3C623400020000000000000000800000000000000000000000000000000000000000000000000080000000000000000000000000000000000000008002000DFF9E
:3C6270000200000000000000000006000000000000000000000000000000000000000000000000400000000000000000000000000000000000000000800025FF06
:3C62AC00008206000000000000880800000000000000000000000000000000000000000000000000000000000000000000000000000000C4160000B0080049FFC4
:3C62E800000006000000000000000000000000000000000000000000000000000000000000000000000000000000000000000000000000000600000000007EFEF2
:3C63240000000600000000000000000000000000000000000000000000000000000000000000000000000000000000000000000000000080000000000200D2FEE5
:3C63600002A006000000000000A040000000000000000000000000000000000000000000000000000000000000000000000000000000008000040080800056FEA1
:3C639C0002000000000000000024000000000000000000000000000000000000000000000000000000000000000000000000000000000090000000010000D5FF3A
:3C63D8000200000000000000000000000000000000000000000000000000000000000000000000000000000000000000000000000000000006000000000029FF59
:3C6414000080000000000000008006000000000000000000000000000000000000000000000000000000000000000000010001000000008000000080000008FE3E
:3C645000000000000000000000000000000000000000000000000000000000000000000000800100000000000000008000800000000000400600004010081CFED7
:3C648C0000C40000000000000000000000000000000000000000000000000000000000000000000000000000000000000000000000000088160000B00800EDFFCE
:3C64C8000000000000000000000000000000000000000000000000000000000000000000000000000000000000000000000000000000000006000000000018FE7C
:3C6504000000000000000000000000000000000000000000000000000000000000000000000000000000000000000000000000000000008000000000000096FE47
:3C654000028000000000000000000000000000000000000000000000000000000000000000000000000000000000000000000000000000C00604008082009AFE39
:3C657C00020200000000000000000000000000000000000000000000000000000000000000000000000000000000000000000000000000A100000001000087FEB8
:3C65B80000800680008000800080008000800080008000800080008000800080008000800080008000800080008000800080008000800080008000800000E9FFB9
:3C65F400020000000000000000000000000000000000000000000000000000000000000000000000000001000000010000000100000000000000000001003EFF28
:3C66300002200600000000000000000000000000000000000000000000000000000000000000000000800000008000000080000000000000060000C010082EFF7B
:3C666C00000000000000000000000000000000000000000000000000000000000000000000000000000000000000000000000000000000000000000000001EFED6
:3C66A800000000000000000000000000000000000000000000000000000000000000002000000000000000000000000000000000010000200000000000000CFE6B
:3C66E400000000000000000000000000000000000000000000000000000000000000000000000000000000000000000000000000000000000000000000001EFE5E
:3C672000000000000000000000000000000000000000000000000000000000000000000000000000000000000000000000000000000000000000000000001EFE21
:3C675C00000000000000000000000000000000000000000000000000000000000000000000000000000000000000000000000000000000200000000002001EFEC3
:3C679800000000000000000000000000000000000000000000000000000000000000000000000000000000000000000000000000000000000000000020000DFF99
:3C67D40002000000000000000000000000000000000000000000000000000000000000000000000000000000010000000000000000000000000000008800AEFF51
:3C6810000000000000000000000000000000000000000000000000000000000000000000000000000100000000000000000004000000000000004008000046FEBB
:3C684C00000000000000000000000000000000000000000000000000000000000000000000000000000000000000020000000000000000040000000410006AFF8D
:3C6888000000000000000000000000000000000000000000000000000000000000000000000004000000000000000000000002000000000000200002000018FE96
:3C68C400001200000000000000400000000000000000000000000000000000000000010004000040000000000000010000000040000000000000000000202EFE74
:3C690000000000000000000000000000000000000000000000000000000000000000000000000000010000000000000000000000000000000000100000000EFF3D
:3C693C00000000000000000000000000000000000000000000000000000000000000000000000000000000000000000000000000000000000000000000001EFE03
:3C697800000000000000000000000000000000000000000000000000000000000000000000000000000000000000000000000000000000000000000000001EFEC7
:3C69B40000000000000000000000000000000000000000000000000000000000000000000000000000000400000000000000000000000000000008000000DAFEC3
:3C69F000000000000000000000200000000000000000000000000000000000000000100000004000000000000000000002004000000010000000400004000EFE59
:3C6A2C00000000000000000000000000000000000000000000000000000000000000000000000000000000000000000000000000000000000000000000001EFE12
:3C6A6800000000000000000000000000000000000000000000000000000000000000000000000000000000000000000000000000000000000000000000001EFED6
:3C6AA400000000000000000000000000000000000000000000000000000000000000000000000000000000000000000000000000000000000000000000001EFE9A
:3C6AE000000000000000000000000000000000000000000000000000000000000000000000000000000000000000000000000000000000000000000000001EFE5E
:3C6B1C000000000000000000000000000000000000000000000000000000000000000000000000000000000000000000000000000000000000000008000016FE21
:3C6B5800000000000000000000000000000000000000000000000000000000000000000000000000000000000000000000000000000000000000000000001EFEE5
:3C6B9400000000000000000000000000000000000000000000000000000000000000000000000000000000000000000000000000000000000000000000001EFEA9
:3C6BD000000000000000000000000000000000000000000000000000000000000000000000000000000000000000000000000000000000000000000000001EFE6D
:3C6C0C00000000000000000000000000000000000000000000000000000000000000000000000000000000000000000000000000000000000000000000001EFE30
:3C6C4800000000000000000000000400000000000000000000000000000000000000000000000000040000000000000000000000040000000000004000005AFE6C
:3C6C8400000000000000000000000000000000000000000000000000000000000000000004000000000000000000000000000000000000000000000000005AFE78
:3C6CC000000000000000000000000000000000000000000000000000000000000000000000000000000000000000000000000000000000000000000000001EFE7C
:3C6CFC00008000000000000000000000000000000000000000000000000000000000000000000000000000000000000000000000000000100000000000009EFF2F
:3C6D3800000000000000000000000000000000000000000000000000000000000000000000000000000000000000000000000000000000000000000000001EFE03
:3C6D7400000000000000000000000000000000000000000000000000000000000000000000000000000000000000000000000000000000000000000000001EFEC7
:3C6DB000000000000000000000000000000000000000000000000000000000000000000400000000000000000000000000000000000000000000001000000AFE8B
:3C6DEC00000001000000000020000000000000000000000000000000000000000000000000000000000000000000000000000000000000000000000000001CFF2F
:3C6E28000000000000000000000000000000000000000000000000000000000000000000000000000000000000000000000000000000800000000004000012FE9A
:3C6E640000000000000000000028000000000000000000000000000000000000000000000000000000000000000000000000000002000000060000000400DEFEE2
:3C6EA0000002000000000000000000000000000000000000000000000000000000000000000000400000000000000000000000100000000800000000000198FFC4
:3C6EDC0002000000000000000000000000000000000000000000000000000000000000840E0000000000000000000000000000000000000000000000000045FFA2
:3C6F18000000000000000000000000000000000000000000000000000000000000000000060000000000000000000000000000000000000000000000000078FEC1
:3C6F540000000000000000000000000000000000000000000000000000000000000000800200000000000000000000000000000000000000000000000000BCFEC5
:3C6F900000000000000000000000000000000000000000000000000000000000000000A0820000000000000000000000000000000000000000000000000094FE11
:3C6FCC0000000000000000000000000000000000000000000000000000000000000000800400000000000000000000000000000000000000000000000000DAFE2D
:3C700800000000000000000000000000000000000000000000000000000000000000000002000000000000000000000000000000000000000000000000003CFE10
:3C704400000000000000000000000000000000000000000000000000000000000000008000000000000000000000000000000000000000000000000000009EFEF4
:3C7080000000000000000000000000000000000000000000000000000000000000000000480000000000000000000000000000000000000000000000000092FEFC
:3C70BC0008000000000000000000000000000000000000000000000000000000000000A206000000000000000000000000000000000000000000000000005AFE90
:3C70F8000000000000000000000000000000000000000000000000000000000000000000060000000000000000000000000000000000000000000000000078FEE0
:3C71340000000000000000000000000000000000000000000000000000000000000000800200000000000000000000000000000000000000000000000000BCFEE3
:3C71700002080000000000000000000000000000000000000000000000000000000000802A000000000000000000000000000000000000000000000000000FFF21
:3C71AC0012000000000000000000000000000000000000000000000000000000000000800000000000000000000000000000000000000000000000000000AFFE68
:3C71E800020000000000000000000000000000000000000000000000000000000000000000000000000000000000000000000000000000000000000000003EFE2D
:3C722400020000000000000000000000000000000000000000000000000000000000008002000000000000000000000000000000000000000000000000008DFF1E
:3C7260000002000000000000000000000000000000000000000000000000000000000000140200000000000000000000000000000000000000000000000079FE63
:3C729C0008000000000000000000000000000000000000000000000000000000000000840E00000000000000000000000000000000000000000000000000F4FE2A
:3C72D80000000000000000000000000000000000000000000000000000000000000000000600000000000000000000000000000000000000000000800000F8FEFE
:3C73140000000000000000000000000000000000000000000000000000000000000000800200000000000000000000000000000000000000000000000000BCFE01
:3C73500002080000000000000000000000000000000000000000000000000000000000C02200000000000000000000000000000000000000000000000000C7FF4F
:3C738C0002000000000000000000000000000000000000000000000000000000000000800000000000000000000000000000000000000000000000000000AFFF95
:3C73C800020000000000000000000000000000000000000000000000000000000000000000000000000000000000000000000000000000000000000000003EFE4B
:3C740400020000000000000000000000000000000000000000000000000000000000008003000000000000000000000000000000000000000000000000008DFE3C
:3C74400008020000000000000000000000000000000000000000000000000000000000801402000000000000000000000000000000000000000000800000F9FEF9
:3C747C0000000000000000000000000000810600000000000000000000000000000080801600000000000000000000000000000080C01600000000000000A8FF3A
:3C74B8000000000000000000000000000000000000000000000000000000000000000000060000000000000000000000000000000000000000000000000078FE1C
:3C74F400000000000000000000000000000006000000000000000000000000000000008002000000000000000000000000000000008006000000000000003CFE14
:3C75300002000000000000000000000000A01608000000000000000000000000000000C022000000000000000000000000000000008020000000000000001BFEC4
:3C756C000200000000000000000000000002160000000000000000000000000000000080000000000000000000000000000000000082000000000000000059FE70
:3C75A80000000000000000000000000000800600000000000000000000000000000000000000000000000000000000000000000000000000000000000000F8FE2B
:3C75E40002000000000000000000000000800400000000000000000000000000000000800300000000000000000001000000000000800600000000000000BFFE1E
:3C7620000200000000000000000000000020020800000000000000000000000000000080140200000000000000800000000000000020060000000000000017FEB1
:3C765C0008000000000000000000000000810600000000000000000000000000000000840E00000000000000000000000000000000A10E000000000000005CFEC8
:3C7698000000000000000000000000000000060000000000000000000000000000000000060000000000000000000000000000000000060000000000000078FE2E
:3C76D4000000000000000000000000000000060000000000000000000000000000000080020000000000000000000000000000000080020000000000000078FEFA
:3C77100002080000000000000000000000A01008000000000000000000000000000000C0820000000000000000000000000000000080820000000000000057FEE2
:3C774C0002000000000000000000000000020C00000000000000000000000000000000800400000000000000000000000000000000800400000000000000E1FF09
:3C778800020000000000000000000000000002000000000000000000000000000000000002000000000000000000000000000000000002000000000000001CFEA3
:3C77C40002000000000000000000000000800600000000000000000000000000000000800000000000000000000000000000000001800000000000000000D9FF28
:3C7800001008000000000000000000000040060400000000000000000000000000000000300000000000000000000000000000800000300000000000000069FEA3
:3C783C0008000000000000000000000000810000000000000000000000000000000000900E0000000000000000000000000000000000000000000000000070FF7A
:3C787800000000000000000000000000000000000000000000000000000000000000000000000000000000000000000000000000000000000000000000001EFEB8
:3C78B400000000000000000000000000000006000000000000000000000000000000008006000000000000000000000000000000000000000000000000009EFE70
:3C78F00002080000000000000000000000A01608000000000000000000000000000000A08600000000000000000000000000000000000000000000000000BFFEB1
:3C792C0002000000000000000000000000010600000000000000000000000000000000A20000000000000000000000000000000000000000000000000000FBFE7B
:3C79680002000000000000000000000000800600000000000000000000000000000000000000000000000000000000000000000000000000000000000000D8FE85
:3C79A400020000000000000000000000008000000000000000000000000000000000008000000000000000000000000000000000000000000000000000002FFF77
:3C79E000500000000000000000000000004006000000000000000000000000000000000006000000000000000000000000000000000000000000000000000BFEC6
:3C7A1C0000000000000000000000000000810600000000000000000000000000000000B00E0000000000000000000000000000000000000000000000000827FEBC
:3C7A58000000000000000000000000000000060000000000000000000000000000000000000000000000000000000000000000000000000000000000000078FE76
:3C7A9400000000000000000000000000000006000000000000000000000000000000008006000000000000000000000000000000000000000000000000009EFE8E
:3C7AD00002000000000000000000000000A01008000000000000000000000000000000808600000000000000000000000000000000000000000000000020D3FEC9
:3C7B0C000200000000000000000000000021140000000000000000000000000000008080000000000000000000000000000000000000000000000000002421FFC2
:3C7B4800000000000000000000000000000002000000000000000000000000000000000000000000000000000000000000000000000000000000000000002DFFD3
:3C7B84000200000000000000000000000080060000000000000000000100010000000080000000000000010000000000000000000000000000000000000059FF62
:3C7BC00002000000000000800100008001000604000000000000008000800000000000400600000000800000000000000000000000000000000000000000AEFF08
:3C7BFC0000000000000000000000000000810000000000000000000000000000000000D00A000000000000821600000000000000000000000000000000004AFF11
:3C7C3800000000000000000000000000000000000000000000000000000000000000000002000000000000000600000000000000000000000000000000003AFED0
:3C7C74000000000000000000000000000000060000000000000000000000000000000080060000000000000006000000000000000000000000000000000098FEAC
:3C7CB00002000000000000000000000000A016080000000000000000000000000000008086000000000000C00601000000000000000000000000000000005DFFAF
:3C7CEC000200000000000000000000000000060000000000000000000000000000000080080000000000000002000000000000000000000000000000000043FF88
:3C7D28000000000000000000000000000080060000000000000000000000000000000000000000000000008004000000000000000000000000000000000074FEA3
:3C7D640002000000000000000000000000800400000000000000000001000000000000800400000000000080060000000000000000000000000000000000B1FFA2
:3C7DA00002000000000000000000000000001204000000000000008000000000000000000284010000000000160800000000000000000000000000800100B1FE3A
:3C7DDC000800000000000000000000000081060000000000000000000000000000000090020000000000008406000000000000000000000000000000000885FE35
:3C7E1800000000000000000000000000000006000000000000000000000000000000000002000000000000000600000000000000000000000000000000005CFEC6
:3C7E540000000000000000000000000000000200000000000000000000000000000000800600000000000000060000000000000000000000000000000000DCFE8A
:3C7E900002080000000000000000000000A01208000000000000000000000000000000C016020000000000C0120800000000000000000000000000000020D7FF4A
:3C7ECC00120000000000000000000000804010000000000000000000000000000000008008000000000000241000000000000000000000000000000000228FFF2C
:3C7F0800020000000000000000000000000006000000000000000000000000000000000000000000000000000400000000000000000000000000000000004DFFE5
:3C7F44000200000000000000000000000080060000000000000000000000000000000080040000000000008006000000010000000000000000000000000083FEED
:3C7F800000080000000000000000008001000602000000000000000000000080010000000204008001000000060100800000000000000000000000800100ACFF79
:3C7FBC0008000000000000000000000000000000000000000000000000000000000000880600000000000000000000000000000000880E0000000000000887FFCF
:3C7FF800000000000000000000000000000000000000000000000000000000000000000000000000000000000000000000000000000000000000000000001EFE31
:3C803400000000000000000000000000000000000000000000000000000000000000008006000000000000000000000000000000008006000000000000001EFEE8
:3C80700002080000000000000000000000000000000000000000000000000000000000C01602000000000000000000000000000000C086000000000000203DFE51
:3C80AC000A0000000000000000000000000000000000000000000000000000000000008400000000000000000000000000000000008100000000000000487FFEC4
:3C80E80002800080008000800080008000800080008000800080008000800080008000800080008000800080008000800080008000800080008000800000AFFFAC
:3C812400020000000000000000000000000000000000000000000000000000000000000000000000000000000000000000000000000000000000000001002FFEEF
:3C8160000004008001000000000000000000000000800100008001800180010000800120060000000000000000000000000000000020060000000080000002FF0C
:3C819C00000000000000000000000000000000000000000000000000000000000000000000000000000000000000000000000000000000000000000000001EFE8B
:3C81D8000000008000000000008000000000000000800000008000800000008000000020000000000000000000000000000000000020008000000080000016FE17
:3C821400000000000000000000000000000200000000000000000000000000000000004000000000000000000000000000000000000000000000000000005CFE92
:3C825000000000000000000000000000000000000000000000000000000000000000000000000000000000000000000000000000000000000000000000001EFED6
:3C828C00000000000000000000000000000000000000000000000000000000000000000000000000000000000000000000000000000000000000000000001EFE9A
:3C82C80000000000000000000000000040000000000000000000000000000000000000800000000000000000000000000000000000000000000000000000DAFEE2
:3C830400000000000000000000000000000000000000000000000000000000000000000000000000000000000000000000000000000000000000000000001EFE21
:3C8340000000000000000000000000000408000000000000000000000000000000000000000000000400000800000000000000000100400000000000000082FE28
:3C837C008000000400000000000000000000000000040000000000000000000000000000000000000000000000000000000000000004000000000000000096FEA5
:3C83B800020000000000000000000000000000000000000000000000000000000000020200000000000000000000000000000000000000000000000000001CFE69
:3C83F400100000000000000000000000000000400000000000000000000000000000000004000000000000000040010000000000000000000000000000000AFFAF
:3C843000000000000000000000000000000000000000000000000000000000000000000000000000000000000000000000000000000000000000000000001EFEF4
:3C846C00001000000000000000000000000000000000000000000000000000000000000000000000000000000000000000000000000002000000000000002CFE98
:3C84A8000000000000000000000000002000000000000400000004000000000000000000001000000000000000000000000000000000000000000000000078FFE9
:3C84E4000042000004000000000000008000002000000000000000000000000000000080010000000000002000010000020000000000000000000000020050FE82
:3C8520000000000000000000000000000000010000000000000000000400040002002048000000000000000000000000000000000002000000000000044070FFF7
:3C855C00000000000000000000000000000000000000000000000000000000000000000000000000000000000000000000000000000000000000000000001EFEC7
:3C859800000000000000000000000000000000000000000000000000000000000000000000000000000000000000000000000000000000000000000000001EFE8B
:3C85D400000000000000000000000000000000000000000000000000000000000000000000000000000000000000000000000000000000000000000000001EFE4F
:3C8610000008000000000000000200000000000000000000000200020000000000000000000100000000000000000000000000000000000000000000000024FEFD
:3C864C00000000000000000000000000000000000000000000000000000000000000000020000000000000000000000000000000200000000000004000007EFEF6
:3C868800000000000000000000000000000000000000000000000000000000000000000000000000000000000000000000000000000000000000000000001EFE9A
:3C86C40000000000000000000000000000000000000000000000000000000000000000000000000000000000000000000000000080000000000000000002B6FE44
:3C870000000000000000000000000000000100000000000000000000000040000000000000000000000000000000000000000000000000000000000000000AFFF3
:3C873C00000000000000000000000000000000000000000000000000000000000000000000000000000000000000000000000000000000000000000000001EFEE5
:3C87780000000000000000000000000000000000000000000000000000000000000000000002000000000000000000000000000000000000000000000800B6FE07
:3C87B400000000000000000000000000000000000000000000000000000000000000000000000000000000000000000000000000000000000000000000045EFE29
:3C87F00000000000000000000000000000000084000000000000000020000000000000000000000000002000000000000000000000000000000000000000F6FE95
:3C882C00000000000000000000000000000000000000000000000000000000000000000000000000000000000000000000000000000000000000000000001EFEF4
:3C88680000800000000000000000000020000000000000000000000000000000000000400000000000000000000000000000000000000000000000000030DEFFE7
:3C88A400000000000000000000000000000000000000000000000000000000000000000000000000000000000000000000000000000000000000000000001EFE7C
:3C88E00000000000000000000000000000400000000000000000000000000000000000000000000000000040000000000000000000000000000000000082B2FEAA
:3C891C004000010000000000200000000000000000000000000000000000000000000000000000000000000000000000000000000000000000000000000418FFA3
:3C8958001000000000000000000000000000002000000000000000001000000000000000000010000000000800000000000000008000000000000000000464FEA5
:3C8994000800000000000000000000000000040000000000000000000000000000000008040000000000000000000000000000000000000000000000000096FEFB
:3C89D0000400000000000000000000000000000800000000000000000000000200000002280000000000000000000000000000000000020200000002000076FEB9
:3C8A0C00100000000000000000000000000000000000000000000000000000000000000000000000000000000000000000000000000000000000000000088FFE89
:3C8A4800000000000000000000000000000000000000000000000000000000000000000000000000000000000000000000000000000000000000000000001EFED6
:3C8A8400000000000000000000000000000000000000000000000000000000000000000000000000000000000000000000000000000000000000000000001EFE9A
:3C8AC0000208000000000000000000000000000000000000000000000000000000000000000000000000000000000000000000000000000000000000002005FF4C
:3C8AFC00020000000000000000000000000000000000000000000000000000000000000000000000000000000000000000000000000000000000000000020FFF2C
:3C8B3800020000000000000000000000000000000000000000000000000000000000000000000000000000000000000000000000000000000000000000002FFFD1
:3C8B7400020000000000000000000000000000000000000000000000000000000000000000000000000000000000000000000000000000000000000000002FFF95
:3C8BB0001008000000000000000000000000000000000000000000000000000000000000000000000000000000000000000000000000000000000000004052FFE0
:3C8BEC000081060000000000000000000000000000000000000000000000000080C00200000000000000000000000000000000000000000000000000000044FF41
:3C8C2800000000000000000000000000000000000000000000000000000000000000020000000000000000000000000000000000000000000000000000003EFED2
:3C8C64000000060000000000000000000000000000000000000000000000000000800200000000000000000000000000000000000000000000000000000050FEFE
:3C8CA00002C0160800000000000000000000000000000000000000000000000000802A00000000000000000000000000000000000000000000000000000093FE7D
:3C8CDC008240060000000000000000000000000000000000000000000000000000801000000000000000000000000000000000000000000000000000000089FE7D
:3C8D180000800600000000000000000000000000000000000000000000000000000000000000000000000000000000000000000000000000000000000000F8FEA3
:3C8D54000280040000000000000000000000000000000000000000000000000000800600000000000000000000000000000000000000000000000000000083FF55
:3C8D900002000A01000000000000000000000000000000000000000000000000000006020000000000000000000000000000000000000000000000000000F7FF9C
:3C8DCC000081060000000000000000000000000000000000000000000000000080C00E00000000000000000000000000000000000000000000000000000815FE7B
:3C8E080000000600000000000000000000000000000000000000000000000000000000000000000000000000000000000000000000000000000000800000F8FEB2
:3C8E44000000060000000000000000000000000000000000000000000000000000800600000000000000000000000000000000000000000000000000000010FE58
:3C8E800002C0100800000000000000000000000000000000000000000000000000802000000000000000000000000000000000000000000000000000002077FEA7
:3C8EBC0002240C00000000000000000000000000000000000000000000000000008200000000000000000000000000000000000000000000000000000022EFFFB6
:3C8EF800000002000000000000000000000000000000000000000000000000000000000000000000000000000000000000000000000000000000000000002DFF10
:3C8F340002800600000000000000000000000000000001000000000000000000008006000000000000000000000000000000000000000000000000000000B1FF42
:3C8F70000200060200000000000000000000000000800000000000000000000000200600000000000000000000000000000000000000000000000080000092FE05
:3C8FAC000281060000000000000000000000000000000000000000000000000080C016000000000000000000000000000000000000000000000000000008B5FFEE
:3C8FE8000000060000000000000000000000000000000000000000000000000000000000000000000000000000000000000000000000000000000000000078FED1
:3C9024000000060000000000000000000000000000000000000000000000000000800600000000000000000000000000000000000000000000000000000010FE76
:3C90600002C0160800000000000000000000000000000000000000000000000000802000000000000000000000000000000000000000000000000000002011FE25
:3C909C0012480600000000000000000000000000000000000000000000000000808000000000000000000000000000000000000000000000000000000024EBFE2B
:3C90D80002800600000000000000000000000000000000000000000000000000000000000000000000000000000000000000000000000000000000000000C9FF0C
:3C91140002800000000000000000000000000000000000000000000000000000008006000000000000000000000001000000000000000100000000000000D7FE40
:3C9150000208060000000000008001000000000000000000000000000000000000200600000000000000000000800000000000000080000000000000000022FF0B
:3C918C0000810600000000000000000000000000000000000000000000A20E0080C00200000000000000000000000000408002000000000000000000000086FFE7
:3C91C800000006000000000000000000000000000000000000000000000006000000020000000000000000000000000000000200000000000000000000003CFE21
:3C9204000000060000000000000000000000000000000000000000000080020000800200000000000000000000000000008002000000000000000000000078FE2C
:3C92400002C010080000000000000000000000000000000000000000008002010080320000000000000000000000000000A03200000000000000000000005FFFB3
:3C927C0002021400000000000000000000000000000000000000000000800400008008000000000000000000000000000080100000000000000000000000ADFE57
:3C92B800000002000000000000000000000000000000000000000000000002000000000000000000000000000000000000000000000000000000000000001EFE5A
:3C92F40002800600000000000000000000000000000000000000000000800000008006000000000000000000000000000080060001000000000000000000BFFF6B
:3C93300002200602000000000000000000000000000000000000000000003000000006020000000000000000000000000000868000000000000000000000B7FEE4
:3C936C0002810000000000000000000000000000000000000000000000000000000000000000000000000000000000000000000000000000000000000000AEFF95
:3C93A800000000000000000000000000000000000000000000000000000000000000000000000000000000000000000000000000000000000000000000001EFE6D
:3C93E4000000060000000000000000000000000000000000000000000000000000000000000000000000000000000000000000000000000000000000000078FED1
:3C94200000C0160800000000000000000000000000000000000000000000000000000000000000000000000000000000000000000000000000000000000039FEFB
:3C945C000200160000000000000000000000000000000000000000000000000000000000000000000000000000000000000000000000000000000000000059FE65
:3C94980002800600000000000000000000000000000000000000000000000000000000000000000000000000000000000000000000000000000000000000D8FE3A
:3C94D40002800400000000000000000000000000000000000000000000000000000000000000000000000000000000000000000000000000000000000000EBFFEC
:3C951000120182000000000000800100000000000000000000000000000000000000000000000000000000000000000000000000000000000000008001000DFF7C
:3C954C000081060000000000000000000000000000000000000000000000000080C00600000000000000000000000000000000000000000000000000000004FF13
:3C9588000000060000000000000000000000000000000000000000000000000000000600000000000000000000000000000000000000000000000000000018FE85
:3C95C4000000020000000000000000000000000000000000000000000000000000800000000000000000000000000000000000000000000000000000000034FEB7
:3C96000002C01208000000000000000000000000000000000000000000000000008008040000000000000000000000000000000000000000000000000000D1FEF7
:3C963C008200000000000000000000000000000000000000000000000000000000B000000000000000000000000000000000000000000000000000000000BDFE05
:3C9678000000060000000000000000000000000000000000000000000000000000000600000000000000000000000000000000000000000000000000000018FE94
:3C96B40002800600000000000000000000000000000001000100000000000000008000000000000000000000000000000000000000000000010001000000D1FF9E
:3C96F00002200E04000000000000008001000000008000800000000000000000000006000000000000000000000000000000000000000080008000000000D1FFB3
:3C972C00008100000000000000000000000000000000000000000000000000000088080000000000000000000000000000000000000080801400000000001AFFC3
:3C976800000000000000000000000000000000000000000000000000000000000000000000000000000000000000000000000000000000000400000000001AFEA9
:3C97A400000006000000000000000000000000000000000000000000000000000000000000000000000000000000000000000000000000000600000000007EFE01
:3C97E00002C0160800000000000000000000000000000000000000000000000000C0000100000000000000000000000000000000000000C00604000000008BFF58
:3C981C0002000E00000000000000000000000000000000000000000000000000002110000000000000000000000000000000000000000000020000000000C1FF0D
:3C985800008006000000000000000000000000000000000000000000000000000080020000000000000000000000000000000000000000800400000000005CFEEE
:3C9894000280040000000000000000000000000000000000000001000000000000800000000000000000010000000000000000000000008002000000010079FE96
:3C98D00002000208000000000000000000000000000000000080000000000000000020000000000000800080010000000000000000800100140800800000A3FFF0
:3C990C0000810600000000C800000000000000000000000000C406000000000000C100000000000000000000000000000000000000004080160000000008ADFFBB
:3C994800000006000000000000000000000000000000000000000600000000000000000000000000000000000000000000000000000000000200000000007CFE5B
:3C998400000002000000000000000000000000000000000000000600000000000000000000000000000000000000000000000000000000000600000000003CFE5F
:3C99C00002C012080000008000000000000000000000000000800600000000000080280000000000000000000000000000000000000000A006040000002033FEE6
:3C99FC004200080000000044000000000000000000000000000000000000000000300000000000000000000000000000000000000000002404000000000493FEB4
:3C9A3800000006000000000006000000000000000000000000000000000000000000000000000000000000000000000000000000000000000200000000000DFFD8
:3C9A74000280060000000080000000000000000000000000008000000000000000800200000000000000000000000000010000000000008004000000000065FEC4
:3C9AB0000220860000000000060000000000000000000000000000000000000000003000000000000000008001000080000000000000008017080000002008FFD5
:3C9AEC0000000000000000000000000000000000000000000000000000880E0080C0060000000000000000000000000000A416000000000000000000000068FE42
:3C9B28000000000000000000000000000000000000000000000000000000000000000600000000000000000000000000000006000000000000000000000078FE7F
:3C9B64000000000000000000000000000000000000000000000000000080060000800000000000000000000000000000008000000000000000000000000078FEC9
:3C9BA00002000000000000000000000000000000000000000000000000C006010080080200000000000000000000000000808000000000000000000000001BFF1C
:3C9BDC000200000000000000000000000000000000000000000000000082000000880000000000000000000000000000008800000000000000000000000025FF95
:3C9C180000800080008000800080008000800080008000800080008000800080008006800080008000800080008000800080068000800080008000800000F8FE0E
:3C9C5400020000000000000000000000000000000000000000000000000000000000000000000000000000000000000000000000000000000000010000003FFF93
:3C9C900002000000008001000080010000800100000000000000000000400680014006000000000000000000000000000040060000000000008000000000BFFE83
:3C9CCC00000000000000000000000000000000000000000000000000000000000000000000000000000000000000000000000000000000000000000000001EFE40
:3C9D0800000000000000000000000000000000000000000000000080002000000020000000800080000000800000000000200000000000000000000000001EFEA3
:3C9D4400000000000000000000000000000000000000000000000000000000000000000000000000000000000000000000000000000000000000000000001EFEC7
:3C9D8000000000000000000000000000000000000000000000000000000000000000000000000000000000000000000000000000000000000000000000001EFE8B
:3C9DBC00000000000000000000000000000000000000000000000000000000000000000000000000000000000000000000000000000000000000000000001EFE4F
:3C9DF8000000020000000000000000000000000000000000000000000000000000000000000000000000000000000000000000000000000000000000008834FE73
:3C9E3400000000000000000000000000000000000000000000000000000000000000000000000000000000000000000000000000000000000000000000001EFED6
:3C9E7000000000000000000000000000000000000000000000000000000000004000000000000000000000000000000000000000010000000000000000004EFE29
:3C9EAC00000000000000000000000000000000000000000000000004000000000000000000000000000000000000000000000000000000000000000000005AFE1E
:3C9EE800000000020000000000000000000002000000000000000000000800000200000800000000000000000000000000001000000000000000020000003FFFD8
:3C9F2400000000400000000000000100000000000000000000000000000000010000000100000000000000000000010000000000000001000040000000005EFF1F
:3C9F600000400000000000000000000000000000000000000000000000000000080000000000000000000000000000000000040000000000000000000080DAFE21
:3C9F9C00000001000000000000000000000000000000000000000000000000000000000000000000000000000000000000000000000000000000000000405AFFEF
:3C9FD8000800000000000400000000000000000000000000000000000000000000000000000000000000000000000000000000000000080002000000000054FEE5
:3CA014000800000000000000000004000000000000000000000000000002000000000002000000000000000002000000000000000000000000000000000098FE68
:3CA05000400000000000000000000000000000000000000000000000000000000000000000000000000000000000000002000000000000000020000000006BFF08
:3CA08C00000000000000000000000000000000000000000000000000000000000000000000000000000000000000000000000000000000000000000000001EFE7C
:3CA0C800000000000000000000000000000000000000000000000000000000000000000000000000000000000000000000000000000000000000000000001EFE40
:3CA10400000000000000000000000000000000000000000000000000000000000001100000000000000000000000000000000000000000000000000000001EFEF2
:3CA14000000000000000000000000000000000000000000000000000000200000000000000000000000000000000000000000000000000000000000000001CFEC7
:3CA17C000000200000000000000000000000000000400000000000000000000000000000000000000000000000000000000000000000000000000000000018FE31
:3CA1B800000000000000000000000000000000000000000000000000000000000000000000000000000000000000000000000000000000000000000000001EFE4F
:3CA1F400000000000000000000000000000000000000000000000000000000000000000000000000000000000000000000000000000000000000000000001EFE13
:3CA23000000200000100000000000000000000000000000000001000000000000001000000000000000000000000000000000000000010004000000000004CFF43
:3CA26C00000000000000000000000000000000000000000000000000000000000000000000000000000000000000000010000000000000000000004000004EFF19
:3CA2A8000000400000000000000000000000000000000000000000000000000000000000000000000000080000000000000000000000000000000000000092FEA2
:3CA2E400000000000000000000000000000000000000000000000000000000000000000000000000000000000000000000000000000000000000000000045EFEDE
:3CA3200000000800000000000000000000000000000000000000000000000000000000000000000000000000000000000000000000000000000020000000B4FE27
:3CA35C004021000000000000010080000000000000000000001000000000000000000008000000000000000000000000002400000000000000000000800088FFA0
:3CA39800008000000000001000000000200000000000000000000000000000000000000000000000000000000000000000000000000000000000000000208EFE2D
:3CA3D400000000000000000000000000000000000000000000000000000000000000000000000000000000000000000000000000000000000000000000001EFE31
:3CA4100000000000000000080000000000000000000000000008000000000000004000000000000000000000000000000000000000000040000000000002F6FE8A
:3CA44C00000000100000000000000000000000000000200020000000000000000002000000000000000000000000000000000000000000200000000000003EFF25
:3CA48800000011000000000000000000000000000000000000000000000000000000000200000000000000001000000000000000000020000000000010440AFFF8
:3CA4C40000000000000000080000000000000000000000000000000000000200002000000000000000000000000000000000000000000000000000000080BEFEF6
:3CA50000800020040000000000000000000000000000000000000000000000000000000000020002000000020000000000000000000000000000000000807EFE79
:3CA53C000000000000000000000000000000000000000000000000000000000000000000000000000000000000000000000000000000000000000000800007FF5D
:3CA57800000000000000000000000000000000000000000000000000000000000000000000000000000000000000000000000000000000000000000000001EFE8B
:3CA5B400000000000000000000000000000000000000000000000000000000000000000000000000000000000000000000000000000000000000000000001EFE4F
:3CA5F000020000000000000000000000000000000000000000000000000000000000000000000000000000000000000000000000000000000000000000406BFF83
:3CA62C00020000000000000000000000000000000000000000000000000000000000000000000000000000000000000000000000000000000000000000288DFF3C
:3CA66800000000000000000000000000000000000000000000000000000000000000000000000000000000000000000000000000000000000000000000000FFFA8
:3CA6A400020000000000000000000000000000000000000000000000000000000000000000000000000000000000000000000000000000000000000000002FFF4A
:3CA6E000020000000000000000000000000000000000000000000000000000000000000000000000000000000000000000000000000000000000000000003EFE00
:3CA71C000000000000000000000000000000000000000000000000000000000000000000000000000000000000000000000000840600000000000000000032FE47
:3CA75800000000000000000000000000000000000000000000000000000000000000000000000000000000000000000000000000000000000000000000001EFEA9
:3CA794000000000000000000000000000000000000000000000000000000000000000000000000000000000000000000000000800600000000000000000076FE8F
:3CA7D0000200000000000000000000000000000000000000000000000000000000000000000000000000000000000000000000A02800000000000000000087FFFD
:3CA80C000200000000000000000000000000000000000000000000000000000000000000000000000000000000000000000000820000000000000000000005FF88
:3CA84800000000000000000000000000000000000000000000000000000000000000000000000000000000000000000000000000000000000000000000001EFEB8
:3CA884000200000001000000000000000000010000000000000000000000000000000000000000000000000000000000000001800600000000000000010047FFC6
:3CA8C000020000800000000000000000008000000000000000000000000000000000000000000000000000000000000000800040060000000000008000004BFFCA
:3CA8FC000000000000000000000000000000000000000000000000000000000000000000000000000000000000000000000000840E000000000000000000B2FEDE
:3CA93800000000000000000000000000000000000000000000000000000000000000000000000000000000000000000000000000000000000000000000001EFEC7
:3CA974000000000000000000000000000000000000000000000000000000000000000000000000000000000000000000000000800600000000000000000076FEAD
:3CA9B0000200000000000000000000000000000000000000000000000000000000000000000000000000000000000000000000A02000000000000000000007FFA3
:3CA9EC000200000000000000000000000000000000000000000000000000000000000000000000000000000000000000000000840000000000000000000063FF47
:3CAA2800000000000000000000000000000000000000000000000000000000000000000000000000000000000000000000000000000000000000000000001EFED6
:3CAA64000200000000000100000000000000000000000000000000000000000000000000000000000000000000000000000000800700000000000000000047FFE6
:3CAAA0000200000000800000000000000000000000000000000000000000000000000000000000000000000000000000000000C0060000000000000000004BFFE8
:3CAADC000000000000000000000000000000000000000000000000000000008102000000008416000000000000000000000000820600000000000000800009FF11
:3CAB1800000000000000000000000000000000000000000000000000000000000200000000000000000000000000000000000000060000000000000000007CFE7F
:3CAB540000000000000000000000000000000000000000000000000000000000060000000080060000000000000000000000008002000000000000000000BEFEFB
:3CAB9000020000000000000000000000000000000000000000000000000000C09600000000A020000000000000000000000000C052000000000000000040D3FE4E
:3CABCC00020000000000000000000000000000000000000000000000000000080600000080C000000000000000000000000000801400000000000000004421FE06
:3CAC080000000000000000000000000000000000000000000000000000000080060000000000000000000000000000000000000002000000000000000000A1FFE8
:3CAC44000200000000000000000000000000000000000000000000000000008000000000008006000000000000000100000000800000000000000000000031FF1B
:3CAC8000020000000000000000000000000000000000000000000000000000200E10000000000600000000000080000000000000200000000000000000002EFF85
:3CACBC00020000000000000000000000000000000000000000000000000080C006000084068406000000000000000000000080C0060000000000000000003CFE80
:3CACF8000000000000000000000000000000000000000000000000000000000006000000000000000000000000000000000000000600000000000000000078FE9E
:3CAD34000000000000000000000000000000000000000000000000000000000006000080068006000000000000000000000000800200000000000000000058FEF9
:3CAD700000000000000000000000000000000000000000000000000000000080920000A030A030000000000000000000000000805200000000000000000051FFD3
:3CADAC00020000000000000000000000000000000000000000000000000000241000008100C100000000000000000000000000800400000000000000000059FE18
:3CADE800020000000000000000000000000000000000000000000000000000000400000000000000000000000000000000000000020000000000000000001AFE0F
:3CAE240000000000000000000000000000000000000000000000000000000080060000800680060000000000000000000000008000000000000000000000E1FF00
:3CAE60000000000000000000000000000000000000000000000000000000000006040020060006000000000000000000000000803100000000000000000037FE9A
:3CAE9C000200000000000000000000000000000000000000000000000000008102000000808016000000000000000000000000A40600000000000000800005FFB1
:3CAED80000800000000000000000000000000000000000000000000000000000020000000000020000000000000000000000000006000000000000000000FEFEB8
:3CAF14000000000000000000000000000000000000000000000000000000000006000000000000000000000000000000000000000000000000000000000018FEE5
:3CAF5000000000000000000000000000000000000000000000000000000000C09600000000A022000000000000000000000000802E00000000000000004053FF6D
:3CAF8C00020000000000000000000000000000000000000000000000000000280E000000002416000000000000000000000080001600000000000000000457FE28
:3CAFC8000200000000000000000000000000000000000000000000000000008006000000008006000000000000000000000000800200000000000000000007FFB7
:3CB004000000000000000000000000000000000000000000000000000000008000000000008006000000000000000000000000800600000000000000000061FF24
:3CB0400000800000000000000000000000000000000000000000000000000000860000000000060200000000000000000000002002040000000000800120B8FF48
:3CB07C00020000000000000000000000000000000000000000000000000000A10600000080800E000000000000000000000000A40E000000000000008000BBFFF5
:3CB0B800000000000000000000000000000000000000000000000000000000000600000000000600000000000000000000000000020000000000000000003EFE12
:3CB0F400000000000000000000000000000000000000000000000000000000000600000000000600000000000000000000000000060000000000000000007EFE92
:3CB13000000000000000000000000000000000000000000000000000000000809200000000A006040000000000000000000000800208000000000000004099FFC5
:3CB16C0002000000000000000000000000000000000000000000000000000044100000000024140000000000000000000000800010000000000000000042A9FEA0
:3CB1A800020000000000000000000000000000000000000000000000000000000400000000000000000000000000000000000000060000000000000000004BFF15
:3CB1E4000000010000000000000000000000000001000000000000000000008006000000008004000000000001000000010000800600000000000000000065FF37
:3CB22000008000000000000000000000000000800000008001000000000000000604000000008600000000800000008000000020460000000000000000007CFF00
:3CB25C000000000000000000000000000000000000000000000000000000008106000000808006000000000000000000000000A40E000000000000008000B1FF47
:3CB29800000000000000000000000000000000000000000000000000000000000600000000000200000000000000000000000000060000000000000000007AFEF4
:3CB2D4000000000000000000000000000000000000000000000000000000000006000000000000000000000000000000000000000000000000000000000018FE22
:3CB31000020000000000000000000000000000000000000000000000000000C09600000000A0320000000000000000000000008026000000000000000040E3FF0F
:3CB34C00020000000000000000000000000000000000000000000000000000000E000000002406000000000000000000000080000E00000000000000000205FFF7
:3CB388000000000000000000000000000000000000000000000000000000008006000000008006000000000000000000000000800200000000000000000027FFD5
:3CB3C4000200000000000000000000000000000000000000000000000000008004000000008006000000000000000100010000800600000001000000000045FF74
:3CB40000020000800100000000000000008001000080010000000000000000000204000000000E010000000000800080000000208200008000000000004098FF7D
:3CB43C000200000000000000000000800E00000000000000000000000000008106C20600808016000000000000000000000000A406000000000000008000A7FF0F
:3CB47800000000000000000000000000060000000000000000000000000000000600060000000600000000000000000000000000020000000000000000003EFE42
:3CB4B4000000000000000000000000000000000000000000000000000000000002800200000006000000000000000000000000000600000000000000000052FE7C
:3CB4F000000000000000000000000080800000000000000000000000000000C09280120400A006040000000000000000000000801208000000000000004071FF44
:3CB52C0002000000000000000000000000000000000000000000000000000001008014000024040000000000000000000000800010000000000000000004D1FFC0
:3CB568000200000000000000000000000000000000000000000000000000000006000200000000000000000000000000000000000600000000000000000069FF2F
:3CB5A4000000000000000000000000800600000000000000000000000000008006800000008004000000000000000000010000800600000000000000000005FED1
:3CB5E000000000800100000000800100060000000000000000000000000000200E0100010000160100000000000000800000002006080000000000000040FAFFF9
:3CB61C000000000000000000000000000000000000000000000000000000000000000000000000000000000000000000000000000000000000000000800007FF6C
:3CB65800000000000000000000000000000000000000000000000000000000000000000000000000000000000000000000000000000000000000000000001EFE9A
:3CB69400000000000000000000000000000000000000000000000000000000000000000000000000000000000000000000000000000000000000000000001EFE5E
:3CB6D000020000000000000000000000000000000000000000000000000000000000000000000000000000000000000000000000000000000000000000406BFF92
:3CB70C00020000000000000000000000000000000000000000000000000000000000000000000000000000000000000000000000000000000000000000013FFFC0
:3CB74800008000800080008000800080008000800080008000800080008000800080008000800080008000800080008000800080008000800080008000008FFF37
:3CB78400020000000000000000000000000000000000000000000000000000000000000000000000000000000000000000000000000000000000000000002FFF59
:3CB7C000020000000000000000000000000000800100000000000000000000000000000000000000000000000000000000000000000000800100008001209CFF0D
:3CB7FC00000000000000000000000000000000000000000000000000000000000000000000000000000000000000000000000000000000000000000000001EFEF5
:3CB838000000000000000000000000000000000000000000008000800080008000A0002000A00000000000800000000000000020000000000000000000009CFE3A
:3CB87400000000000000000000000000000000000000000000000000000000000000000000000000000000000000000000000000000000000000000000001EFE7C
:3CB8B000000000000000000000000000000000000000000000000000000000000000000000000000000000000000000000000000000000000000000000001EFE40
:3CB8EC00000000000000000000000000000000000000000000000000000000000000000000000000000000000000000000000000000000000000000000001EFE04
:3CB928000000000000000000000000000000000000000000000000000000000000000000000000000000000000000000000000000000000000000000008096FECF
:3CB964000000000000000000000002000000000000000000000000000000002010000000100004000000000000000100000010800040000000000000000072FF1F
:3CB9A0000000000000000000000000000000000002000000000000000000400000000000000000000000000000000000000000080000000000000000000090FE93
:3CB9DC00000000000000000000000000000000000000000000000000000000000000000000000000000000000000000000000000000000000000000000001EFE13
:3CBA1800000000000000000000000000000000000000000000000000000000000000000000000000000000000000000000000000000000000000000000000FFFE4
:3CBA5400000000000000000000000000000000000000000000000000000000000000000000000000000000000000000000000000000000000000000000001EFE9A
:3CBA9000000000000000000000000000000000000000000000000000000000004000000004000000000000000000000000000000000000000000000000001AFE1E
:3CBACC00000000000000000000000000000000000000000000000000000000000200000000010000000000000000000000000000010000000000000000303EFFCD
:3CBB080002000000020000000000000020000000000000000000000000008000000000000000810000000000000000000000000000000000040000000002A2FF35
:3CBB4400000000000000000000000000000000000000000000000000000000000000000000000000000000000000000000000000000000000000000000001EFEA9
:3CBB80000000000000000000000000000000000000000000000000000000400001200000002010000000000000000000020000200000000000000000840056FFFD
:3CBBBC00000000000000000000000000000000000000000000000000000000000000000000000000000000000000000000000000000000000000000000001EFE31
:3CBBF80000000008000000000000000000000000000000000000000000000000000000000000000000000000000000000000000004000000000000000000DEFE29
:3CBC3400000000000000000000000000000000000000000000000000000000000000000000000000000000000000000000000000000000000000000000001EFEB8
:3CBC7000000000000000000000000000000000000000000000000000000000020000000000020000000000020000000000000000000000000000000000003EFE56
:3CBCAC0000000000004000000000000000000000000000000000000000000000000000000000000000000000000000000000004020800000000000000000BCFE82
:3CBCE800000000000000000000000000000000000000000000000000000000000000000000002004000000000000000050000000000000000000000000006EFF3F
:3CBD2400000000000000000000000000000800000000000000000000000000000000800000000000000000000000000000000000000000000000008000023EFE9D
:3CBD6000000000001000000000000000000000000000000000000000000000100010000000000000000000000000000000000000000000001000000000000EFE5B
:3CBD9C00000000000000000000000000000000000000000000000000000000000000000000000000000000000000000000000000000000000000000000001EFE4F
:3CBDD800000000000000000000000000000008002000000000000000000080004100000000400000000000002000000000000000000000000000000000080AFFD5
:3CBE140000000000000000000000000000000000000000000000000000000000000000000000000000000000000000000008000010200000000000080004F6FFB9
:3CBE5000000000000000000000000000000000000000000000000000000000400000000000000000000000000000000000000000000000000000000000004BFF2C
:3CBE8C00000000000000000000000010000000000000000000000000000000000000000000000000000000000000000000000000000000002000200020000EFFFD
:3CBEC8000000200000000000000000000000000000000000000000000000000000108000000000080000000000000000000000000000000000000000005048FEF0
:3CBF0400000000010000000000000000000000000000000000000000000000000000004000400000000000000000000000000040000000001000000000010EFE23
:3CBF40000000000000000000000000000000000000000800000000000000000000000000200000000000000000000000000020400000010000000000001838FEEE
:3CBF7C00000000000000000000000000000000000000000020000000000000000000000000000020000000000000000000000010000000000000000000044EFFE8
:3CBFB8000000000000000000000000000000000000000000000000000000004000020000000000000000000000001000000000000000000000000000000438FFC0
:3CBFF40000000000000000000000000800000000000000000000000000000000000800000200000000000000000000000000000004000000000000000028DEFEF7
:3CC030000000000000000000000000000000000000000000000200020002000000020000000002000000000000000000000000000200000000000000009096FFA3
:3CC06C00000000000000000000000000000000000000000000000000000000000000000000000080040000000400040000000000000000008000800000001AFEF4
:3CC0A80000000000000000000000000000000000000000000000000000000000000000000000000000800000008000000480040000000000008000800000D6FE00
:3CC0E40000000400040004800000008000800480040000000480040000000000000000000000048004800000048004000480040000000000008000800000D6FE98
:3CC120000000008000800000048004000400000000800480000000800480048004800480048000000000048000000080000000800480048004C004C000001AFE13
:3CC15C0000000480048004800480048004800480048004800480048004800480048004800480048004800480048004800480048004800480448004A8000076FEDF
:3CC1980000000400040004800000008000800480040000000480040000000000000000000000048004800000048004000480040000000000008000800000D6FEE3
:3CC1D400000000800080000004800400040000000080048000000080048004800480048004800000000004800000008000000080048004800480048000005EFE9B
:3CC2100000000080008000000480040004000000008004800000008004800480048004800480000000000480000000800000008004800480042004000000D4FEC8
:02C24C00FFFFF2
:00000001FF
